 usbfn

 Timestamp is 4da293b4 (Mon Apr 11 17:37:56 2011)

 Preferred load address is 10000000

 Start         Length     Name                   Class
 0001:00000000 00000004H .CRT$XCA                CODE
 0001:00000004 00000004H .CRT$XCU                CODE
 0001:00000008 00000004H .CRT$XCZ                CODE
 0001:0000000c 00000004H .CRT$XIA                CODE
 0001:00000010 00000004H .CRT$XIZ                CODE
 0001:00000014 00000004H .CRT$XPA                CODE
 0001:00000018 00000004H .CRT$XPZ                CODE
 0001:0000001c 00000004H .CRT$XTA                CODE
 0001:00000020 00000004H .CRT$XTZ                CODE
 0001:00000030 00000610H .rdata                  CODE
 0001:00000640 00000022H .rdata$debug            CODE
 0001:00000664 0000f154H .text                   CODE
 0001:0000f7b8 00000004H .text$yc                CODE
 0001:0000f7bc 0000000cH .text$yd                CODE
 0001:0000f7c8 00000108H .xdata                  CODE
 0001:0000f8d0 0000003cH .idata$2                CODE
 0001:0000f90c 00000014H .idata$3                CODE
 0001:0000f920 00000190H .idata$4                CODE
 0001:0000fab0 00000068H .idata$6                CODE
 0001:0000fb20 000000f6H .edata                  CODE
 0002:00000000 00000190H .idata$5                DATA
 0002:00000190 00000014H .data                   DATA
 0002:000001c0 0000007cH .bss                    DATA
 0003:00000000 00000c28H .pdata                  DATA

  Address         Publics by Value              Rva+Base       Lib:Object

 0000:00000000       ___safe_se_handler_table   00000000     <absolute>
 0000:00000000       ___safe_se_handler_count   00000000     <absolute>
 0001:00000000       __xc_a                     10001000     corelib0:crt0init.obj
 0001:00000008       __xc_z                     10001008     corelib0:crt0init.obj
 0001:0000000c       __xi_a                     1000100c     corelib0:crt0init.obj
 0001:00000010       __xi_z                     10001010     corelib0:crt0init.obj
 0001:00000014       __xp_a                     10001014     corelib0:crt0init.obj
 0001:00000018       __xp_z                     10001018     corelib0:crt0init.obj
 0001:0000001c       __xt_a                     1000101c     corelib0:crt0init.obj
 0001:00000020       __xt_z                     10001020     corelib0:crt0init.obj
 0001:0000004c       ??_C@_1CC@BJPGGDNC@?$AAU?$AAS?$AAB?$AA_?$AAC?$AAL?$AAO?$AAC?$AAK?$AA_?$AAG?$AAA?$AAT?$AAI?$AAN?$AAG?$AA?$AA@ 1000104c     i_usbclock.obj
 0001:00000070       ??_7CPipeBase@@6B@         10001070     usb_ufnmddbase_common_topaz_v1:pipe.obj
 0001:00000090       ??_7CStaticPipe@@6B@       10001090     usb_ufnmddbase_common_topaz_v1:pipe.obj
 0001:000000b0       ??_7CDynamicPipe@@6B@      100010b0     usb_ufnmddbase_common_topaz_v1:pipe.obj
 0001:000000d0       ??_7CUfnBusDevice@@6B@     100010d0     usb_ufnmddbase_common_topaz_v1:ufnbus.obj
 0001:000000f8       ??_C@_1BK@BFIEKNFP@?$AAF?$AAr?$AAi?$AAe?$AAn?$AAd?$AAl?$AAy?$AAN?$AAa?$AAm?$AAe?$AA?$AA@ 100010f8     usb_ufnmddbase_common_topaz_v1:ufnbus.obj
 0001:00000118       ??_7CUfnBus@@6B@           10001118     usb_ufnmddbase_common_topaz_v1:ufnbus.obj
 0001:00000180       ??_C@_1M@LLKDCKCI@?$AAU?$AAS?$AAB?$AAF?$AAN?$AA?$AA@ 10001180     usb_ufnmddbase_common_topaz_v1:ufnbus.obj
 0001:0000018c       ??_C@_1BA@FGOFGFHE@?$AA?$CF?$AAs?$AA_?$AA?$CF?$AAd?$AA_?$AA0?$AA?$AA@ 1000118c     usb_ufnmddbase_common_topaz_v1:ufnbus.obj
 0001:0000019c       ??_C@_1DK@HJDLAGJ@?$AA?2?$AAD?$AAr?$AAi?$AAv?$AAe?$AAr?$AAs?$AA?2?$AAU?$AAS?$AAB?$AA?2?$AAF?$AAu?$AAn?$AAc?$AAt?$AAi?$AAo?$AAn?$AAD?$AAr?$AAi?$AAv?$AAe?$AAr?$AAs?$AA?$AA@ 1000119c     usb_ufnmddbase_common_topaz_v1:ufnbus.obj
 0001:000001d8       ??_C@_1M@DFKENGJN@?$AA?$CF?$AAs?$AA?2?$AA?$CF?$AAs?$AA?$AA@ 100011d8     usb_ufnmddbase_common_topaz_v1:ufnbus.obj
 0001:000001e4       ??_C@_1CI@MGKPCHDE@?$AAD?$AAe?$AAf?$AAa?$AAu?$AAl?$AAt?$AAC?$AAl?$AAi?$AAe?$AAn?$AAt?$AAD?$AAr?$AAi?$AAv?$AAe?$AAr?$AA?$AA@ 100011e4     usb_ufnmddbase_common_topaz_v1:ufnbus.obj
 0001:0000020c       ??_C@_1CC@COLLGMBE@?$AAD?$AAe?$AAf?$AAa?$AAu?$AAl?$AAt?$AAC?$AAl?$AAi?$AAe?$AAn?$AAt?$AAK?$AAe?$AAy?$AA?$AA@ 1000120c     usb_ufnmddbase_common_topaz_v1:ufnbus.obj
 0001:00000230       ??_C@_17DJMMGLBL@?$AAD?$AAl?$AAl?$AA?$AA@ 10001230     usb_ufnmddbase_common_topaz_v1:ufnbus.obj
 0001:00000238       ??_7SVSTree@@6B@           10001238     ceosutil:utilmemf.obj
 0001:00000248       ??_7CRefObject@@6B@        10001248     defbuslib:DefBus.obj
 0001:0000024c       ??_C@_1M@JLADBBAF@?$AAE?$AAn?$AAt?$AAr?$AAy?$AA?$AA@ 1000124c     defbuslib:DefBus.obj
 0001:00000258       ??_7DefaultBusDriver@@6B@  10001258     defbuslib:DefBus.obj
 0001:000002bc       ??_C@_1BA@HABJOAEE@?$AAU?$AAN?$AAK?$AAN?$AAO?$AAW?$AAN?$AA?$AA@ 100012bc     defbuslib:DefBus.obj
 0001:000002cc       ??_C@_1M@KCNCFNNL@?$AA$?$AAb?$AAu?$AAs?$AA?2?$AA?$AA@ 100012cc     defbuslib:DefBus.obj
 0001:000002d8       ??_C@_1M@OAJFFPML@?$AAF?$AAl?$AAa?$AAg?$AAs?$AA?$AA@ 100012d8     defbuslib:DefBus.obj
 0001:000002e4       ??_C@_1M@PJMPBMAL@?$AAO?$AAr?$AAd?$AAe?$AAr?$AA?$AA@ 100012e4     defbuslib:DefBus.obj
 0001:000002f0       ??_C@_1BA@KDCCGFJM@?$AAB?$AAu?$AAs?$AAN?$AAa?$AAm?$AAe?$AA?$AA@ 100012f0     defbuslib:DefBus.obj
 0001:00000300       ??_C@_1BI@CDNKGHCP@?$AA?$CF?$AAs?$AA_?$AA?$CF?$AAd?$AA_?$AA?$CF?$AAd?$AA_?$AA?$CF?$AAd?$AA?$AA@ 10001300     defbuslib:DefBus.obj
 0001:00000318       ??_C@_1BE@PMMIAJMN@?$AAB?$AAu?$AAs?$AAP?$AAa?$AAr?$AAe?$AAn?$AAt?$AA?$AA@ 10001318     defbuslib:DefBus.obj
 0001:0000032c       ??_C@_1BM@MHMIAMLB@?$AAI?$AAn?$AAt?$AAe?$AAr?$AAf?$AAa?$AAc?$AAe?$AAT?$AAy?$AAp?$AAe?$AA?$AA@ 1000132c     defbuslib:DefBus.obj
 0001:00000348       ??_7DeviceFolder@@6B@      10001348     defbuslib:DefBus.obj
 0001:00000370       ??_C@_1BC@GDFGLIEL@?$AAO?$AAT?$AAG?$AAG?$AAr?$AAo?$AAu?$AAp?$AA?$AA@ 10001370     usb_usbfn_mx25_topaz_v1:i_pdd.obj
 0001:00000384       ??_C@_1BG@HHFAGDDC@?$AAO?$AAT?$AAG?$AAS?$AAu?$AAp?$AAp?$AAo?$AAr?$AAt?$AA?$AA@ 10001384     usb_usbfn_mx25_topaz_v1:i_pdd.obj
 0001:0000039c       ??_C@_1BI@BHLBGEOK@?$AAP?$AAr?$AAi?$AAo?$AAr?$AAi?$AAt?$AAy?$AA2?$AA5?$AA6?$AA?$AA@ 1000139c     usb_usbfn_mx25_topaz_v1:i_pdd.obj
 0001:000003b4       ??_C@_17DJGGJCGD@?$AAI?$AAr?$AAq?$AA?$AA@ 100013b4     usb_usbfn_mx25_topaz_v1:i_pdd.obj
 0001:000003bc       ??_C@_1O@LBBNFMDB@?$AAM?$AAe?$AAm?$AAL?$AAe?$AAn?$AA?$AA@ 100013bc     usb_usbfn_mx25_topaz_v1:i_pdd.obj
 0001:000003cc       ??_C@_1BA@INLDIDEN@?$AAM?$AAe?$AAm?$AAB?$AAa?$AAs?$AAe?$AA?$AA@ 100013cc     usb_usbfn_mx25_topaz_v1:i_pdd.obj
 0001:00000470       ??_C@_1BM@LGGJJGMB@?$AAP?$AAr?$AAi?$AAm?$AAe?$AAF?$AAZ?$AAL?$AAT?$AA?3?$AA?5?$AA?$CF?$AAs?$AA?$AA@ 10001470     usb_usbfn_mx25_topaz_v1:i_pdd.obj
 0001:0000048c       ??_C@_17HCEMPBGG@?$AAO?$AAU?$AAT?$AA?$AA@ 1000148c     usb_usbfn_mx25_topaz_v1:i_pdd.obj
 0001:00000494       ??_C@_15BNKBCKPG@?$AAI?$AAN?$AA?$AA@ 10001494     usb_usbfn_mx25_topaz_v1:i_pdd.obj
 0001:000004a0       ??_C@_1EA@GOCNCOIC@?$AAI?$AAs?$AAs?$AAu?$AAe?$AAT?$AAr?$AAa?$AAn?$AAs?$AAf?$AAe?$AAr?$AA?3?$AA?5?$AA?$CF?$AAs?$AA?5?$AAw?$AAi?$AAt?$AAh?$AA?5?$AA?$CF?$AAd?$AA?5?$AAb?$AAy?$AAt?$AAe?$AAs?$AA?$AA@ 100014a0     usb_usbfn_mx25_topaz_v1:i_pdd.obj
 0001:000004e0       ??_C@_1DA@JMEFNML@?$AAA?$AAb?$AAo?$AAr?$AAt?$AAT?$AAr?$AAa?$AAn?$AAs?$AAf?$AAe?$AAr?$AA?5?$AA?$CI?$AA?$CF?$AAs?$AA?5?$AAE?$AAP?$AA?$CF?$AAd?$AA?$CJ?$AA?$AA@ 100014e0     usb_usbfn_mx25_topaz_v1:i_pdd.obj
 0001:00000510       ??_C@_19CIJIHAKK@?$AAN?$AAU?$AAL?$AAL?$AA?$AA@ 10001510     usb_usbfn_mx25_topaz_v1:i_pdd.obj
 0001:0000051c       ??_C@_1CA@HMLLGPGC@?$AA?9?$AAS?$AAe?$AAn?$AAd?$AAC?$AAS?$AAH?$AA?5?$AA?$CI?$AAE?$AAP?$AA?$CF?$AAd?$AA?$CJ?$AA?$AA@ 1000151c     usb_usbfn_mx25_topaz_v1:i_pdd.obj
 0001:0000053c       ??_C@_1CA@DFPEHIFN@?$AA?$CL?$AAS?$AAe?$AAn?$AAd?$AAC?$AAS?$AAH?$AA?5?$AA?$CI?$AAE?$AAP?$AA?$CF?$AAd?$AA?$CJ?$AA?$AA@ 1000153c     usb_usbfn_mx25_topaz_v1:i_pdd.obj
 0001:0000055c       ??_C@_1CI@HKDMKLGF@?$AAD?$AAe?$AAt?$AAa?$AAc?$AAh?$AA?3?$AA?5?$AAP?$AAO?$AAR?$AAT?$AAS?$AAC?$AA?5?$AA0?$AAx?$AA?$CF?$AAx?$AA?$AA@ 1000155c     usb_usbfn_mx25_topaz_v1:i_pdd.obj
 0001:00000584       ??_C@_1O@BJIMCIMK@?$AAR?$AAe?$AAs?$AAu?$AAm?$AAe?$AA?$AA@ 10001584     usb_usbfn_mx25_topaz_v1:i_pdd.obj
 0001:00000594       ??_C@_1BE@JNFMNJIM@?$AAI?$AAn?$AAt?$AAr?$AA?3?$AAD?$AAo?$AAn?$AAe?$AA?$AA@ 10001594     usb_usbfn_mx25_topaz_v1:i_pdd.obj
 0001:000005a8       ??_C@_1EE@JAFGGGNF@?$AAI?$AAn?$AAt?$AAr?$AA?3?$AAU?$AAI?$AA?5?$AAS?$AAE?$AAT?$AAU?$AAP?$AAS?$AAT?$AAA?$AAT?$AA?5?$AA?$CF?$AAx?$AA?5?$AAE?$AAN?$AAD?$AAP?$AAT?$AAC?$AAO?$AAM?$AAP?$AA?5?$AA?$CF@ 100015a8     usb_usbfn_mx25_topaz_v1:i_pdd.obj
 0001:000005ec       ??_C@_1BC@MCOFDLFC@?$AAI?$AAn?$AAt?$AAr?$AA?3?$AAS?$AAL?$AAI?$AA?$AA@ 100015ec     usb_usbfn_mx25_topaz_v1:i_pdd.obj
 0001:00000600       ??_C@_1BO@EGKDOEEI@?$AAI?$AAn?$AAt?$AAr?$AA?3?$AAS?$AAi?$AAg?$AAn?$AAa?$AAl?$AAl?$AAe?$AAd?$AA?$AA@ 10001600     usb_usbfn_mx25_topaz_v1:i_pdd.obj
 0001:00000620       ??_C@_1BA@EKAPLICF@?$AAU?$AAS?$AAB?$AAF?$AAu?$AAn?$AAc?$AA?$AA@ 10001620     usb_usbfn_os_mx25_topaz_v1:i_os.obj
 0001:00000630       ??_C@_1BA@JAHEEJIA@?$AAU?$AAS?$AAB?$AAX?$AAC?$AAV?$AAR?$AA?$AA@ 10001630     usb_usbfn_os_mx25_topaz_v1:i_os.obj
 0001:00000664       BSPGetUSBControllerType    10001664 f   hwinit.obj
 0001:00000afc       HardwareInitialize         10001afc f   hwinit.obj
 0001:00000ba4       BSPUsbResetPHY             10001ba4 f   hwinit.obj
 0001:00000bb4       USBClockGatingLock         10001bb4 f   i_usbclock.obj
 0001:00000bf0       BSPUSBClockCreateFileMapping 10001bf0 f   i_usbclock.obj
 0001:00000c90       BSPUSBClockDeleteFileMapping 10001c90 f   i_usbclock.obj
 0001:00000cd0       BSPUSBClockSwitch          10001cd0 f   i_usbclock.obj
 0001:00000dc4       USBClockInit               10001dc4 f   i_usbclock.obj
 0001:00000dcc       PowerDownSchemeExist       10001dcc f   i_usbutils.obj
 0001:00000e28       BSPUsbXvrEnableVBUSIntr    10001e28 f   i_usbutils.obj
 0001:00000e44       BSPUsbSetBusConfig         10001e44 f   i_usbutils.obj
 0001:00000e54       BSPUSBInterruptControl     10001e54 f   i_usbutils.obj
 0001:00000e98       BSPPhyShowDevDiscon        10001e98 f   i_usbutils.obj
 0001:00000ea0       BSPUsbSetCurrentLimitation 10001ea0 f   i_usbutils.obj
 0001:00000ea4       ?SetChildDevicePowerState@CUfnBus@@QAAHW4_CEDEVICE_POWER_STATE@@@Z 10001ea4 f i usb_ufnmddbase_common_topaz_v1:ufnmdd.obj
 0001:00000ee8       ?FindPipe@@YAPAVCPipeBase@@PAUUFN_MDD_CONTEXT@@K@Z 10001ee8 f   usb_ufnmddbase_common_topaz_v1:ufnmdd.obj
 0001:00000f4c       ?UfnMdd_Start@@YAKPAXP6AH0KK@Z0PAPAX@Z 10001f4c f   usb_ufnmddbase_common_topaz_v1:ufnmdd.obj
 0001:00001100       ?DoStop@@YAKPAUUFN_MDD_CONTEXT@@@Z 10002100 f   usb_ufnmddbase_common_topaz_v1:ufnmdd.obj
 0001:000011d8       ?UfnMdd_Stop@@YAKPAX@Z     100021d8 f   usb_ufnmddbase_common_topaz_v1:ufnmdd.obj
 0001:00001210       ?DoDeregisterDevice@@YAKPAUUFN_MDD_CONTEXT@@@Z 10002210 f   usb_ufnmddbase_common_topaz_v1:ufnmdd.obj
 0001:000012a8       ?UfnMdd_DeregisterDevice@@YAKPAX@Z 100022a8 f   usb_ufnmddbase_common_topaz_v1:ufnmdd.obj
 0001:00001300       ?UfnMdd_OpenPipe@@YAKPAXKPAPAX@Z 10002300 f   usb_ufnmddbase_common_topaz_v1:ufnmdd.obj
 0001:00001408       ?UfnMdd_ClosePipe@@YAKPAX0@Z 10002408 f   usb_ufnmddbase_common_topaz_v1:ufnmdd.obj
 0001:00001484       ?UfnMdd_GetTransferStatus@@YAKPAX0PAK1@Z 10002484 f   usb_ufnmddbase_common_topaz_v1:ufnmdd.obj
 0001:0000150c       ?UfnMdd_AbortTransfer@@YAKPAX0@Z 1000250c f   usb_ufnmddbase_common_topaz_v1:ufnmdd.obj
 0001:00001578       ?UfnMdd_CloseTransfer@@YAKPAX0@Z 10002578 f   usb_ufnmddbase_common_topaz_v1:ufnmdd.obj
 0001:000015d8       ?UfnMdd_IssueTransfer@@YAKPAX0P6AK0@Z0KK0K0PAPAX@Z 100025d8 f   usb_ufnmddbase_common_topaz_v1:ufnmdd.obj
 0001:000016a8       ?UfnMdd_StallPipe@@YAKPAX0@Z 100026a8 f   usb_ufnmddbase_common_topaz_v1:ufnmdd.obj
 0001:000016fc       ?UfnMdd_ClearPipeStall@@YAKPAX0@Z 100026fc f   usb_ufnmddbase_common_topaz_v1:ufnmdd.obj
 0001:00001750       ?UfnMdd_InitiateRemoteWakeup@@YAKPAX@Z 10002750 f   usb_ufnmddbase_common_topaz_v1:ufnmdd.obj
 0001:000017a0       ?UfnMdd_SendControlStatusHandshake@@YAKPAX@Z 100027a0 f   usb_ufnmddbase_common_topaz_v1:ufnmdd.obj
 0001:0000190c       UFN_PreClose               1000290c f   usb_ufnmddbase_common_topaz_v1:ufnmdd.obj
 0001:00001930       UFN_PowerDown              10002930 f   usb_ufnmddbase_common_topaz_v1:ufnmdd.obj
 0001:0000195c       UFN_PowerUp                1000295c f   usb_ufnmddbase_common_topaz_v1:ufnmdd.obj
 0001:00001990       UFN_IOControl              10002990 f   usb_ufnmddbase_common_topaz_v1:ufnmdd.obj
 0001:00001b1c       ?SendDeviceNotification@@YAHP6AHPAXKK@Z0KK@Z 10002b1c f   usb_ufnmddbase_common_topaz_v1:ufnmdd.obj
 0001:00001b78       ?_Buynode@?$list@KVallocator@ce@@@ce@@IAAPAU?$_ListNode@K@list_impl@2@PAU342@@Z 10002b78 f i usb_ufnmddbase_common_topaz_v1:ufnmdd.obj
 0001:00001bc4       ?Open@CReg@@QAAHPAUHKEY__@@PBGK@Z 10002bc4 f i usb_ufnmddbase_common_topaz_v1:ufnmdd.obj
 0001:00001c34       ?UfnMdd_RegisterDevice@@YAKPAXPAU_USB_DEVICE_DESCRIPTOR@@PAU_UFN_CONFIGURATION@@12PBU_UFN_STRING_SET@@K@Z 10002c34 f   usb_ufnmddbase_common_topaz_v1:ufnmdd.obj
 0001:00001ed4       ?GetClientFunctions@@YAKPAU_UFN_FUNCTIONS@@@Z 10002ed4 f   usb_ufnmddbase_common_topaz_v1:ufnmdd.obj
 0001:00001f88       ?get_lock@?$singleton@V?$free_list@$0GE@Vallocator@ce@@@ce@@$03V?$static_allocator@V?$free_list@$0GE@Vallocator@ce@@@ce@@$03@2@@ce@@KAAAVcritical_section@2@XZ 10002f88 f i usb_ufnmddbase_common_topaz_v1:ufnmdd.obj
 0001:00001fdc       ?erase@?$list@KVallocator@ce@@@ce@@QAA?AV?$iterator@K@list_impl@2@V342@@Z 10002fdc f i usb_ufnmddbase_common_topaz_v1:ufnmdd.obj
 0001:00002038       ?erase@?$list@KVallocator@ce@@@ce@@QAA?AV?$iterator@K@list_impl@2@V342@0@Z 10003038 f i usb_ufnmddbase_common_topaz_v1:ufnmdd.obj
 0001:00002090       ??$for_each@V?$iterator@K@list_impl@ce@@P6AHK@Z@std@@YAP6AHK@ZV?$iterator@K@list_impl@ce@@0P6AHK@Z@Z 10003090 f i usb_ufnmddbase_common_topaz_v1:ufnmdd.obj
 0001:000020d4       ?DeinitializeClass@?$CTransferQueue@VCUfnMddTransfer@@@@SAXXZ 100030d4 f i usb_ufnmddbase_common_topaz_v1:ufnmdd.obj
 0001:00002114       ??$insert@K@?$list@KVallocator@ce@@@ce@@QAA?AV?$iterator@K@list_impl@1@V231@ABK@Z 10003114 f i usb_ufnmddbase_common_topaz_v1:ufnmdd.obj
 0001:0000215c       UFN_PreDeinit              1000315c f   usb_ufnmddbase_common_topaz_v1:ufnmdd.obj
 0001:000021c4       DllEntry                   100031c4 f   usb_ufnmddbase_common_topaz_v1:ufnmdd.obj
 0001:00002234       ?remove@?$list@KVallocator@ce@@@ce@@QAAXABK@Z 10003234 f i usb_ufnmddbase_common_topaz_v1:ufnmdd.obj
 0001:0000228c       ??$Deinit@P6AHK@Z@COpenList@@QAAXP6AHK@Z@Z 1000328c f i usb_ufnmddbase_common_topaz_v1:ufnmdd.obj
 0001:000022d8       ?AddContext@COpenList@@QAA_NK@Z 100032d8 f i usb_ufnmddbase_common_topaz_v1:ufnmdd.obj
 0001:0000233c       UFN_Open                   1000333c f   usb_ufnmddbase_common_topaz_v1:ufnmdd.obj
 0001:000023cc       UFN_Close                  100033cc f   usb_ufnmddbase_common_topaz_v1:ufnmdd.obj
 0001:00002534       UFN_Init                   10003534 f   usb_ufnmddbase_common_topaz_v1:ufnmdd.obj
 0001:0000274c       UFN_Deinit                 1000374c f   usb_ufnmddbase_common_topaz_v1:ufnmdd.obj
 0001:00002794       ?GetInterfaceClass@CConfiguration@@QAAPAVCInterface@@KK@Z 10003794 f i usb_ufnmddbase_common_topaz_v1:pipe.obj
 0001:000027e4       ?GetConfigurationClass@CDevice@@QBAPAVCConfiguration@@K@Z 100037e4 f i usb_ufnmddbase_common_topaz_v1:pipe.obj
 0001:00002834       ?OwningInterface@CStaticPipe@@UBAKW4_UFN_BUS_SPEED@@K@Z 10003834 f   usb_ufnmddbase_common_topaz_v1:pipe.obj
 0001:00002844       ?IsPartOfInterface@CStaticPipe@@UBAHW4_UFN_BUS_SPEED@@KK@Z 10003844 f   usb_ufnmddbase_common_topaz_v1:pipe.obj
 0001:00002894       ?GetEndpointDescriptor@CStaticPipe@@UBAPAU_USB_ENDPOINT_DESCRIPTOR@@W4_UFN_BUS_SPEED@@@Z 10003894 f   usb_ufnmddbase_common_topaz_v1:pipe.obj
 0001:000028a4       ?Reset@CStaticPipe@@UAAXXZ 100038a4 f   usb_ufnmddbase_common_topaz_v1:pipe.obj
 0001:000028ec       ?IsReserved@CStaticPipe@@UBAHW4_UFN_BUS_SPEED@@KKK@Z 100038ec f   usb_ufnmddbase_common_topaz_v1:pipe.obj
 0001:00002900       ?Reserve@CStaticPipe@@UAAXW4_UFN_BUS_SPEED@@HKKKPAU_USB_ENDPOINT_DESCRIPTOR@@@Z 10003900 f   usb_ufnmddbase_common_topaz_v1:pipe.obj
 0001:000029ac       ?GetEndpointAddress@CPipeBase@@QBAKXZ 100039ac f   usb_ufnmddbase_common_topaz_v1:pipe.obj
 0001:000029f4       ?GetTransferStatus@CPipeBase@@SAKPBVCUfnMddTransfer@@PAK1@Z 100039f4 f   usb_ufnmddbase_common_topaz_v1:pipe.obj
 0001:00002a40       ?Stall@CPipeBase@@QAAKXZ   10003a40 f   usb_ufnmddbase_common_topaz_v1:pipe.obj
 0001:00002a88       ?ClearStall@CPipeBase@@QAAKXZ 10003a88 f   usb_ufnmddbase_common_topaz_v1:pipe.obj
 0001:00002ad0       ?SendControlStatusHandshake@CPipeBase@@QAAKXZ 10003ad0 f   usb_ufnmddbase_common_topaz_v1:pipe.obj
 0001:00002b10       ?ValidatePipeHandle@CPipeBase@@SAKPBV1@@Z 10003b10 f   usb_ufnmddbase_common_topaz_v1:pipe.obj
 0001:00002b80       ?_InitializeDescr@?$fixed_block_allocator@$07@ce@@IBA_NI@Z 10003b80 f i usb_ufnmddbase_common_topaz_v1:pipe.obj
 0001:00002be0       ?_Buynode@?$list@U?$pair@KK@std@@Vallocator@ce@@@ce@@IAAPAU?$_ListNode@U?$pair@KK@std@@@list_impl@2@PAU342@@Z 10003be0 f i usb_ufnmddbase_common_topaz_v1:pipe.obj
 0001:00002c2c       ?_Buynode@?$list@U?$pair@KPAU_USB_ENDPOINT_DESCRIPTOR@@@std@@Vallocator@ce@@@ce@@IAAPAU?$_ListNode@U?$pair@KPAU_USB_ENDPOINT_DESCRIPTOR@@@std@@@list_impl@2@PAU342@@Z 10003c2c f i usb_ufnmddbase_common_topaz_v1:pipe.obj
 0001:00002c78       ?_InitializeDescr@?$fixed_block_allocator@$0BE@@ce@@IBA_NI@Z 10003c78 f i usb_ufnmddbase_common_topaz_v1:pipe.obj
 0001:00002cd8       ?GetInterface@CDescriptors@@QAAKW4_UFN_BUS_SPEED@@KPAK@Z 10003cd8 f i usb_ufnmddbase_common_topaz_v1:pipe.obj
 0001:00002d20       ?IsReserved@CPipeBase@@UBAHW4_UFN_BUS_SPEED@@@Z 10003d20 f   usb_ufnmddbase_common_topaz_v1:pipe.obj
 0001:00002dc0       ?Open@CPipeBase@@QAAKW4_UFN_BUS_SPEED@@PAU_USB_ENDPOINT_DESCRIPTOR@@@Z 10003dc0 f   usb_ufnmddbase_common_topaz_v1:pipe.obj
 0001:00002ed0       ?push@?$interlocked_stack@PAXV?$fixed_block_allocator@$07@ce@@@@QAA_NABQAX@Z 10003ed0 f i usb_ufnmddbase_common_topaz_v1:pipe.obj
 0001:00002f50       ?pop@?$interlocked_stack@PAXV?$fixed_block_allocator@$07@ce@@@@QAA_NAAPAX@Z 10003f50 f i usb_ufnmddbase_common_topaz_v1:pipe.obj
 0001:00002fbc       ?erase@?$list@U?$pair@KK@std@@Vallocator@ce@@@ce@@QAA?AV?$iterator@U?$pair@KK@std@@@list_impl@2@V342@@Z 10003fbc f i usb_ufnmddbase_common_topaz_v1:pipe.obj
 0001:00003018       ?erase@?$list@U?$pair@KK@std@@Vallocator@ce@@@ce@@QAA?AV?$iterator@U?$pair@KK@std@@@list_impl@2@V342@0@Z 10004018 f i usb_ufnmddbase_common_topaz_v1:pipe.obj
 0001:00003070       ?erase@?$list@U?$pair@KPAU_USB_ENDPOINT_DESCRIPTOR@@@std@@Vallocator@ce@@@ce@@QAA?AV?$iterator@U?$pair@KPAU_USB_ENDPOINT_DESCRIPTOR@@@std@@@list_impl@2@V342@@Z 10004070 f i usb_ufnmddbase_common_topaz_v1:pipe.obj
 0001:000030cc       ?erase@?$list@U?$pair@KPAU_USB_ENDPOINT_DESCRIPTOR@@@std@@Vallocator@ce@@@ce@@QAA?AV?$iterator@U?$pair@KPAU_USB_ENDPOINT_DESCRIPTOR@@@std@@@list_impl@2@V342@0@Z 100040cc f i usb_ufnmddbase_common_topaz_v1:pipe.obj
 0001:00003124       ??$insert@U?$pair@KK@std@@@?$list@U?$pair@KK@std@@Vallocator@ce@@@ce@@QAA?AV?$iterator@U?$pair@KK@std@@@list_impl@1@V231@ABU?$pair@KK@std@@@Z 10004124 f i usb_ufnmddbase_common_topaz_v1:pipe.obj
 0001:00003174       ?deallocate@?$CFreePool@$03V?$fixed_block_allocator@$07@ce@@Utransfer_funcs@@@@QAAXPAXI@Z 10004174 f i usb_ufnmddbase_common_topaz_v1:pipe.obj
 0001:00003210       ?erase@?$hash@V?$hash_map_traits@KKU?$hash_traits@K@ce@@Vallocator@2@@details@ce@@@details@ce@@QAA?AV?$iterator@U?$pair@KK@std@@@list_impl@3@V453@@Z 10004210 f i usb_ufnmddbase_common_topaz_v1:pipe.obj
 0001:0000327c       ?clear@?$hash@V?$hash_map_traits@KKU?$hash_traits@K@ce@@Vallocator@2@@details@ce@@@details@ce@@QAAXXZ 1000427c f i usb_ufnmddbase_common_topaz_v1:pipe.obj
 0001:000032cc       ?find@?$hash@V?$hash_map_traits@KKU?$hash_traits@K@ce@@Vallocator@2@@details@ce@@@details@ce@@QBA?AV?$const_iterator@U?$pair@KK@std@@@list_impl@3@ABK@Z 100042cc f i usb_ufnmddbase_common_topaz_v1:pipe.obj
 0001:00003350       ?find@?$hash@V?$hash_map_traits@KPAU_USB_ENDPOINT_DESCRIPTOR@@U?$hash_traits@K@ce@@Vallocator@3@@details@ce@@@details@ce@@QBA?AV?$const_iterator@U?$pair@KPAU_USB_ENDPOINT_DESCRIPTOR@@@std@@@list_impl@3@ABK@Z 10004350 f i usb_ufnmddbase_common_topaz_v1:pipe.obj
 0001:000033d4       ?PopulateCache@?$CFreePool@$03V?$fixed_block_allocator@$07@ce@@Utransfer_funcs@@@@IAAXXZ 100043d4 f i usb_ufnmddbase_common_topaz_v1:pipe.obj
 0001:00003478       ??0?$list@PAVCUfnMddTransfer@@V?$fixed_block_allocator@$0BE@@ce@@@ce@@QAA@ABV?$fixed_block_allocator@$0BE@@1@@Z 10004478 f i usb_ufnmddbase_common_topaz_v1:pipe.obj
 0001:000034b8       ?erase@?$list@PAVCUfnMddTransfer@@V?$fixed_block_allocator@$0BE@@ce@@@ce@@QAA?AV?$iterator@PAVCUfnMddTransfer@@@list_impl@2@V342@@Z 100044b8 f i usb_ufnmddbase_common_topaz_v1:pipe.obj
 0001:00003524       ?erase@?$vector@U?$pair@V?$iterator@U?$pair@KK@std@@@list_impl@ce@@I@std@@Vallocator@ce@@U?$exponential_growth@$09@4@@ce@@QAAPAU?$pair@V?$iterator@U?$pair@KK@std@@@list_impl@ce@@I@std@@PAU34@0@Z 10004524 f i usb_ufnmddbase_common_topaz_v1:pipe.obj
 0001:00003588       ?erase@?$vector@U?$pair@V?$iterator@U?$pair@KPAU_USB_ENDPOINT_DESCRIPTOR@@@std@@@list_impl@ce@@I@std@@Vallocator@ce@@U?$exponential_growth@$09@4@@ce@@QAAPAU?$pair@V?$iterator@U?$pair@KPAU_USB_ENDPOINT_DESCRIPTOR@@@std@@@list_impl@ce@@I@std@@PAU34@0@Z 10004588 f i usb_ufnmddbase_common_topaz_v1:pipe.obj
 0001:000035ec       ?erase@?$list@PAVCUfnMddTransfer@@V?$fixed_block_allocator@$0BE@@ce@@@ce@@QAA?AV?$iterator@PAVCUfnMddTransfer@@@list_impl@2@V342@0@Z 100045ec f i usb_ufnmddbase_common_topaz_v1:pipe.obj
 0001:00003644       ?erase@?$vector@U?$pair@V?$iterator@U?$pair@KK@std@@@list_impl@ce@@I@std@@V?$reference_allocator@Vallocator@ce@@@details@ce@@U?$exponential_growth@$09@5@@ce@@QAAPAU?$pair@V?$iterator@U?$pair@KK@std@@@list_impl@ce@@I@std@@PAU34@0@Z 10004644 f i usb_ufnmddbase_common_topaz_v1:pipe.obj
 0001:000036a8       ?erase@?$vector@U?$pair@V?$iterator@U?$pair@KPAU_USB_ENDPOINT_DESCRIPTOR@@@std@@@list_impl@ce@@I@std@@V?$reference_allocator@Vallocator@ce@@@details@ce@@U?$exponential_growth@$09@5@@ce@@QAAPAU?$pair@V?$iterator@U?$pair@KPAU_USB_ENDPOINT_DESCRIPTOR@@@std@@@list_impl@ce@@I@std@@PAU34@0@Z 100046a8 f i usb_ufnmddbase_common_topaz_v1:pipe.obj
 0001:0000370c       ??$insert@U?$pair@KPAU_USB_ENDPOINT_DESCRIPTOR@@@std@@@?$list@U?$pair@KPAU_USB_ENDPOINT_DESCRIPTOR@@@std@@Vallocator@ce@@@ce@@QAA?AV?$iterator@U?$pair@KPAU_USB_ENDPOINT_DESCRIPTOR@@@std@@@list_impl@1@V231@ABU?$pair@KPAU_USB_ENDPOINT_DESCRIPTOR@@@std@@@Z 1000470c f i usb_ufnmddbase_common_topaz_v1:pipe.obj
 0001:0000375c       ?_Buynode@?$list@PAVCUfnMddTransfer@@V?$fixed_block_allocator@$0BE@@ce@@@ce@@IAAPAU?$_ListNode@PAVCUfnMddTransfer@@@list_impl@2@PAU342@@Z 1000475c f i usb_ufnmddbase_common_topaz_v1:pipe.obj
 0001:000037c4       ?OwningInterface@CDynamicPipe@@UBAKW4_UFN_BUS_SPEED@@K@Z 100047c4 f   usb_ufnmddbase_common_topaz_v1:pipe.obj
 0001:00003830       ?IsPartOfInterface@CDynamicPipe@@UBAHW4_UFN_BUS_SPEED@@KK@Z 10004830 f   usb_ufnmddbase_common_topaz_v1:pipe.obj
 0001:000038c0       ?IsReserved@CDynamicPipe@@UBAHW4_UFN_BUS_SPEED@@KKK@Z 100048c0 f   usb_ufnmddbase_common_topaz_v1:pipe.obj
 0001:000039a8       ?GetEndpointDescriptor@CDynamicPipe@@UBAPAU_USB_ENDPOINT_DESCRIPTOR@@W4_UFN_BUS_SPEED@@@Z 100049a8 f   usb_ufnmddbase_common_topaz_v1:pipe.obj
 0001:00003a90       ?FreeTransfer@CPipeBase@@QAAXPAVCUfnMddTransfer@@@Z 10004a90 f   usb_ufnmddbase_common_topaz_v1:pipe.obj
 0001:00003a9c       ?allocate@?$CFreePool@$03V?$fixed_block_allocator@$07@ce@@Utransfer_funcs@@@@QAAPAXI@Z 10004a9c f i usb_ufnmddbase_common_topaz_v1:pipe.obj
 0001:00003b78       ?erase@?$hash@V?$hash_map_traits@KPAU_USB_ENDPOINT_DESCRIPTOR@@U?$hash_traits@K@ce@@Vallocator@3@@details@ce@@@details@ce@@QAA?AV?$iterator@U?$pair@KPAU_USB_ENDPOINT_DESCRIPTOR@@@std@@@list_impl@3@V453@@Z 10004b78 f i usb_ufnmddbase_common_topaz_v1:pipe.obj
 0001:00003be4       ?clear@?$hash@V?$hash_map_traits@KPAU_USB_ENDPOINT_DESCRIPTOR@@U?$hash_traits@K@ce@@Vallocator@3@@details@ce@@@details@ce@@QAAXXZ 10004be4 f i usb_ufnmddbase_common_topaz_v1:pipe.obj
 0001:00003c34       ??$insert@PAVCUfnMddTransfer@@@?$list@PAVCUfnMddTransfer@@V?$fixed_block_allocator@$0BE@@ce@@@ce@@QAA?AV?$iterator@PAVCUfnMddTransfer@@@list_impl@1@V231@ABQAVCUfnMddTransfer@@@Z 10004c34 f i usb_ufnmddbase_common_topaz_v1:pipe.obj
 0001:00003c7c       ?Reset@CDynamicPipe@@UAAXXZ 10004c7c f   usb_ufnmddbase_common_topaz_v1:pipe.obj
 0001:00003cc0       ??1?$list@PAVCUfnMddTransfer@@V?$fixed_block_allocator@$0BE@@ce@@@ce@@QAA@XZ 10004cc0 f i usb_ufnmddbase_common_topaz_v1:pipe.obj
 0001:00003d14       ??1?$hash@V?$hash_map_traits@KKU?$hash_traits@K@ce@@Vallocator@2@@details@ce@@@details@ce@@QAA@XZ 10004d14 f i usb_ufnmddbase_common_topaz_v1:pipe.obj
 0001:00003d54       ??1?$hash@V?$hash_map_traits@KPAU_USB_ENDPOINT_DESCRIPTOR@@U?$hash_traits@K@ce@@Vallocator@3@@details@ce@@@details@ce@@QAA@XZ 10004d54 f i usb_ufnmddbase_common_topaz_v1:pipe.obj
 0001:00003d94       ?TransferComplete@CPipeBase@@QAAKPAVCUfnMddTransfer@@H@Z 10004d94 f   usb_ufnmddbase_common_topaz_v1:pipe.obj
 0001:00003e7c       ?PushBack@?$CTransferQueue@VCUfnMddTransfer@@@@QAAKPAVCUfnMddTransfer@@@Z 10004e7c f i usb_ufnmddbase_common_topaz_v1:pipe.obj
 0001:00003ec0       ?_Insert_dispatch@?$vector@U?$pair@V?$iterator@U?$pair@KK@std@@@list_impl@ce@@I@std@@Vallocator@ce@@U?$exponential_growth@$09@4@@ce@@AAA_NPAU?$pair@V?$iterator@U?$pair@KK@std@@@list_impl@ce@@I@std@@IABU34@ABUtrue_type@detail@2@@Z 10004ec0 f i usb_ufnmddbase_common_topaz_v1:pipe.obj
 0001:00004108       ?_Insert_dispatch@?$vector@U?$pair@V?$iterator@U?$pair@KPAU_USB_ENDPOINT_DESCRIPTOR@@@std@@@list_impl@ce@@I@std@@Vallocator@ce@@U?$exponential_growth@$09@4@@ce@@AAA_NPAU?$pair@V?$iterator@U?$pair@KPAU_USB_ENDPOINT_DESCRIPTOR@@@std@@@list_impl@ce@@I@std@@IABU34@ABUtrue_type@detail@2@@Z 10005108 f i usb_ufnmddbase_common_topaz_v1:pipe.obj
 0001:00004350       ??0CPipeBase@@QAA@KPAU_UFN_PDD_INTERFACE_INFO@@PAVCFreeTransferList@@PAUUFN_MDD_CONTEXT@@@Z 10005350 f   usb_ufnmddbase_common_topaz_v1:pipe.obj
 0001:000043b8       ??0CStaticPipe@@QAA@KPAU_UFN_PDD_INTERFACE_INFO@@PAVCFreeTransferList@@PAUUFN_MDD_CONTEXT@@@Z 100053b8 f   usb_ufnmddbase_common_topaz_v1:pipe.obj
 0001:000043f0       ??1CDynamicPipe@@UAA@XZ    100053f0 f   usb_ufnmddbase_common_topaz_v1:pipe.obj
 0001:00004450       ?IssueTransfer@CPipeBase@@QAAKP6AKPAX@Z0KK0KPAPAVCUfnMddTransfer@@0@Z 10005450 f   usb_ufnmddbase_common_topaz_v1:pipe.obj
 0001:00004668       ?AbortTransfer@CPipeBase@@QAAKPAVCUfnMddTransfer@@@Z 10005668 f   usb_ufnmddbase_common_topaz_v1:pipe.obj
 0001:000046f4       ?CloseTransfer@CPipeBase@@QAAKPAVCUfnMddTransfer@@@Z 100056f4 f   usb_ufnmddbase_common_topaz_v1:pipe.obj
 0001:0000473c       ??_GCPipeBase@@UAAPAXI@Z   1000573c f i usb_ufnmddbase_common_topaz_v1:pipe.obj
 0001:0000473c       ??_ECPipeBase@@UAAPAXI@Z   1000573c f i usb_ufnmddbase_common_topaz_v1:pipe.obj
 0001:00004774       ??_ECStaticPipe@@UAAPAXI@Z 10005774 f i usb_ufnmddbase_common_topaz_v1:pipe.obj
 0001:00004774       ??_GCStaticPipe@@UAAPAXI@Z 10005774 f i usb_ufnmddbase_common_topaz_v1:pipe.obj
 0001:000047ac       ??0CDynamicPipe@@QAA@KPAU_UFN_PDD_INTERFACE_INFO@@PAVCFreeTransferList@@PAUUFN_MDD_CONTEXT@@@Z 100057ac f   usb_ufnmddbase_common_topaz_v1:pipe.obj
 0001:00004908       ??_GCDynamicPipe@@UAAPAXI@Z 10005908 f i usb_ufnmddbase_common_topaz_v1:pipe.obj
 0001:00004908       ??_ECDynamicPipe@@UAAPAXI@Z 10005908 f i usb_ufnmddbase_common_topaz_v1:pipe.obj
 0001:0000492c       ?AbortAllTransfers@CPipeBase@@QAAXXZ 1000592c f   usb_ufnmddbase_common_topaz_v1:pipe.obj
 0001:0000496c       ?resize@?$vector@U?$pair@V?$iterator@U?$pair@KK@std@@@list_impl@ce@@I@std@@Vallocator@ce@@U?$exponential_growth@$09@4@@ce@@QAA_NIABU?$pair@V?$iterator@U?$pair@KK@std@@@list_impl@ce@@I@std@@@Z 1000596c f i usb_ufnmddbase_common_topaz_v1:pipe.obj
 0001:000049c8       ?resize@?$vector@U?$pair@V?$iterator@U?$pair@KPAU_USB_ENDPOINT_DESCRIPTOR@@@std@@@list_impl@ce@@I@std@@Vallocator@ce@@U?$exponential_growth@$09@4@@ce@@QAA_NIABU?$pair@V?$iterator@U?$pair@KPAU_USB_ENDPOINT_DESCRIPTOR@@@std@@@list_impl@ce@@I@std@@@Z 100059c8 f i usb_ufnmddbase_common_topaz_v1:pipe.obj
 0001:00004a24       ?Close@CPipeBase@@QAAKXZ   10005a24 f   usb_ufnmddbase_common_topaz_v1:pipe.obj
 0001:00004a84       ?_ready@?$hash@V?$hash_map_traits@KKU?$hash_traits@K@ce@@Vallocator@2@@details@ce@@@details@ce@@IAA_NXZ 10005a84 f i usb_ufnmddbase_common_topaz_v1:pipe.obj
 0001:00004ae4       ?_ready@?$hash@V?$hash_map_traits@KPAU_USB_ENDPOINT_DESCRIPTOR@@U?$hash_traits@K@ce@@Vallocator@3@@details@ce@@@details@ce@@IAA_NXZ 10005ae4 f i usb_ufnmddbase_common_topaz_v1:pipe.obj
 0001:00004b44       ?insert@?$hash@V?$hash_map_traits@KKU?$hash_traits@K@ce@@Vallocator@2@@details@ce@@@details@ce@@QAA?AV?$iterator@U?$pair@KK@std@@@list_impl@3@ABU?$pair@KK@std@@@Z 10005b44 f i usb_ufnmddbase_common_topaz_v1:pipe.obj
 0001:00004c00       ?find@?$hash@V?$hash_map_traits@KKU?$hash_traits@K@ce@@Vallocator@2@@details@ce@@@details@ce@@QAA?AV?$iterator@U?$pair@KK@std@@@list_impl@3@ABK@Z 10005c00 f i usb_ufnmddbase_common_topaz_v1:pipe.obj
 0001:00004c78       ?insert@?$hash@V?$hash_map_traits@KPAU_USB_ENDPOINT_DESCRIPTOR@@U?$hash_traits@K@ce@@Vallocator@3@@details@ce@@@details@ce@@QAA?AV?$iterator@U?$pair@KPAU_USB_ENDPOINT_DESCRIPTOR@@@std@@@list_impl@3@ABU?$pair@KPAU_USB_ENDPOINT_DESCRIPTOR@@@std@@@Z 10005c78 f i usb_ufnmddbase_common_topaz_v1:pipe.obj
 0001:00004d34       ?find@?$hash@V?$hash_map_traits@KPAU_USB_ENDPOINT_DESCRIPTOR@@U?$hash_traits@K@ce@@Vallocator@3@@details@ce@@@details@ce@@QAA?AV?$iterator@U?$pair@KPAU_USB_ENDPOINT_DESCRIPTOR@@@std@@@list_impl@3@ABK@Z 10005d34 f i usb_ufnmddbase_common_topaz_v1:pipe.obj
 0001:00004dac       ?Reserve@CDynamicPipe@@UAAXW4_UFN_BUS_SPEED@@HKKKPAU_USB_ENDPOINT_DESCRIPTOR@@@Z 10005dac f   usb_ufnmddbase_common_topaz_v1:pipe.obj
 0001:00004ff8       ?ValidateDescriptor@CDescriptors@@SAKPAU_USB_DEVICE_DESCRIPTOR@@PAU_UFN_CONFIGURATION@@01PBU_UFN_STRING_SET@@K@Z 10005ff8 f   usb_ufnmddbase_common_topaz_v1:descript.obj
 0001:000050c0       ?RegisterDevice@CDescriptors@@QAAKPAUUFN_MDD_CONTEXT@@@Z 100060c0 f   usb_ufnmddbase_common_topaz_v1:descript.obj
 0001:0000524c       ?GetDeviceDescriptor@CDescriptors@@QAAPBU_USB_DEVICE_DESCRIPTOR@@W4_UFN_BUS_SPEED@@@Z 1000624c f   usb_ufnmddbase_common_topaz_v1:descript.obj
 0001:00005264       ?CloneStrings@CDescriptors@@SAKPBU_UFN_STRING_SET@@KPAPAU2@@Z 10006264 f   usb_ufnmddbase_common_topaz_v1:descript.obj
 0001:000053d4       ??_I@YAXPAXIHP6AX0@Z@Z     100063d4 f i usb_ufnmddbase_common_topaz_v1:descript.obj
 0001:00005404       ?ValidateDescriptor@CConfiguration@@SAKW4_UFN_BUS_SPEED@@PAU_UFN_CONFIGURATION@@@Z 10006404 f   usb_ufnmddbase_common_topaz_v1:descript.obj
 0001:0000544c       ?FreeUfnConfigTree@CConfiguration@@SAXPAU_UFN_CONFIGURATION@@@Z 1000644c f   usb_ufnmddbase_common_topaz_v1:descript.obj
 0001:00005508       ?ValidateDescriptor@CInterface@@SAKW4_UFN_BUS_SPEED@@PAU_UFN_INTERFACE@@@Z 10006508 f   usb_ufnmddbase_common_topaz_v1:descript.obj
 0001:00005550       ??1CMddEndpoint@@QAA@XZ    10006550 f   usb_ufnmddbase_common_topaz_v1:descript.obj
 0001:00005554       ?IsSupportable@CMddEndpoint@@QAAKPAUUFN_MDD_CONTEXT@@W4_UFN_BUS_SPEED@@EEE@Z 10006554 f   usb_ufnmddbase_common_topaz_v1:descript.obj
 0001:00005658       ?ValidatePacketSize@CMddEndpoint@@CAHW4_UFN_BUS_SPEED@@PAU_USB_ENDPOINT_DESCRIPTOR@@@Z 10006658 f   usb_ufnmddbase_common_topaz_v1:descript.obj
 0001:00005740       ?Serialize@CMddEndpoint@@QAAKPAEKPAK@Z 10006740 f   usb_ufnmddbase_common_topaz_v1:descript.obj
 0001:000057c4       ?InitializeEndpointZeroDescriptor@CMddEndpoint@@SAXEPAU_USB_ENDPOINT_DESCRIPTOR@@@Z 100067c4 f   usb_ufnmddbase_common_topaz_v1:descript.obj
 0001:000057e0       ?ProcessGetDescriptor@CDescriptors@@QAA?AW4CONTROL_RESPONSE@@W4_UFN_BUS_SPEED@@U_USB_DEVICE_REQUEST@@KHPAPAXPAK@Z 100067e0 f   usb_ufnmddbase_common_topaz_v1:descript.obj
 0001:00005a48       ?CopyUfnConfigTree@CConfiguration@@SAKPAU_UFN_CONFIGURATION@@0@Z 10006a48 f   usb_ufnmddbase_common_topaz_v1:descript.obj
 0001:00005ce0       ?Init@CInterface@@QAAKW4_UFN_BUS_SPEED@@PAU_UFN_INTERFACE@@@Z 10006ce0 f   usb_ufnmddbase_common_topaz_v1:descript.obj
 0001:00005da0       ?Serialize@CInterface@@QAAKPAEKPAK@Z 10006da0 f   usb_ufnmddbase_common_topaz_v1:descript.obj
 0001:00005e94       ?IsSupportable@CInterface@@QAAKPAUUFN_MDD_CONTEXT@@W4_UFN_BUS_SPEED@@E@Z 10006e94 f   usb_ufnmddbase_common_topaz_v1:descript.obj
 0001:00005f28       ?ValidateDescriptor@CMddEndpoint@@SAKW4_UFN_BUS_SPEED@@PAU_UFN_ENDPOINT@@@Z 10006f28 f   usb_ufnmddbase_common_topaz_v1:descript.obj
 0001:00005f74       ?IsEndpointZeroSupportable@CMddEndpoint@@SAKPAUUFN_MDD_CONTEXT@@W4_UFN_BUS_SPEED@@PAU_USB_DEVICE_DESCRIPTOR@@@Z 10006f74 f   usb_ufnmddbase_common_topaz_v1:descript.obj
 0001:00006000       ?Clone@CDevice@@QAAKPAV1@@Z 10007000 f   usb_ufnmddbase_common_topaz_v1:descript.obj
 0001:0000609c       ?Init@CConfiguration@@QAAKW4_UFN_BUS_SPEED@@PAU_UFN_CONFIGURATION@@@Z 1000709c f   usb_ufnmddbase_common_topaz_v1:descript.obj
 0001:00006180       ?IsSupportable@CConfiguration@@QAAKPAUUFN_MDD_CONTEXT@@W4_UFN_BUS_SPEED@@PAU_USB_DEVICE_DESCRIPTOR@@@Z 10007180 f   usb_ufnmddbase_common_topaz_v1:descript.obj
 0001:00006284       ?Serialize@CConfiguration@@QAAKPAEKPAK@Z 10007284 f   usb_ufnmddbase_common_topaz_v1:descript.obj
 0001:00006380       ?GenerateTotalConfigDescriptor@CConfiguration@@QAAKXZ 10007380 f   usb_ufnmddbase_common_topaz_v1:descript.obj
 0001:000063fc       ?ValidateDescriptorAndChildren@CInterface@@SAKW4_UFN_BUS_SPEED@@PAU_UFN_INTERFACE@@@Z 100073fc f   usb_ufnmddbase_common_topaz_v1:descript.obj
 0001:00006450       ?Init@CDevice@@QAAKW4_UFN_BUS_SPEED@@PAU_USB_DEVICE_DESCRIPTOR@@PAU_UFN_CONFIGURATION@@@Z 10007450 f   usb_ufnmddbase_common_topaz_v1:descript.obj
 0001:0000652c       ?GenerateTotalConfigDescriptors@CDevice@@QAAKXZ 1000752c f   usb_ufnmddbase_common_topaz_v1:descript.obj
 0001:0000657c       ?IsSupportable@CDevice@@QAAKPAUUFN_MDD_CONTEXT@@W4_UFN_BUS_SPEED@@@Z 1000757c f   usb_ufnmddbase_common_topaz_v1:descript.obj
 0001:000065f8       ??_ECInterface@@QAAPAXI@Z  100075f8 f i usb_ufnmddbase_common_topaz_v1:descript.obj
 0001:00006694       ?ValidateDescriptorAndChildren@CConfiguration@@SAKW4_UFN_BUS_SPEED@@PAU_UFN_CONFIGURATION@@@Z 10007694 f   usb_ufnmddbase_common_topaz_v1:descript.obj
 0001:00006734       ?Init@CDescriptors@@QAAKPAU_USB_DEVICE_DESCRIPTOR@@PAU_UFN_CONFIGURATION@@01PBU_UFN_STRING_SET@@K@Z 10007734 f   usb_ufnmddbase_common_topaz_v1:descript.obj
 0001:00006780       ?IsSupportable@CDescriptors@@QAAKPAUUFN_MDD_CONTEXT@@@Z 10007780 f   usb_ufnmddbase_common_topaz_v1:descript.obj
 0001:00006834       ?ValidateDescriptorAndChildren@CDevice@@SAKW4_UFN_BUS_SPEED@@PAU_USB_DEVICE_DESCRIPTOR@@PAU_UFN_CONFIGURATION@@@Z 10007834 f   usb_ufnmddbase_common_topaz_v1:descript.obj
 0001:000068d8       ??1CConfiguration@@QAA@XZ  100078d8 f   usb_ufnmddbase_common_topaz_v1:descript.obj
 0001:00006908       ?ValidateDescriptorAndChildren@CDescriptors@@SAKPAU_USB_DEVICE_DESCRIPTOR@@PAU_UFN_CONFIGURATION@@01PBU_UFN_STRING_SET@@K@Z 10007908 f   usb_ufnmddbase_common_topaz_v1:descript.obj
 0001:00006968       ??_ECConfiguration@@QAAPAXI@Z 10007968 f i usb_ufnmddbase_common_topaz_v1:descript.obj
 0001:000069d8       ??1CDevice@@QAA@XZ         100079d8 f   usb_ufnmddbase_common_topaz_v1:descript.obj
 0001:00006a48       ??0CDescriptors@@QAA@XZ    10007a48 f   usb_ufnmddbase_common_topaz_v1:descript.obj
 0001:00006ab8       ??1CDescriptors@@QAA@XZ    10007ab8 f   usb_ufnmddbase_common_topaz_v1:descript.obj
 0001:00006ae4       ?Clone@CDescriptors@@QAAKPAPAV1@@Z 10007ae4 f   usb_ufnmddbase_common_topaz_v1:descript.obj
 0001:00006c08       ?AddRef@CUfnMddTransfer@@QAAXXZ 10007c08 f   usb_ufnmddbase_common_topaz_v1:transfer.obj
 0001:00006c10       ?Release@CUfnMddTransfer@@QAAXXZ 10007c10 f   usb_ufnmddbase_common_topaz_v1:transfer.obj
 0001:00006c34       ?Init@CUfnMddTransfer@@QAAXKPAXKK0P6AK0@Z0PAVCPipeBase@@@Z 10007c34 f   usb_ufnmddbase_common_topaz_v1:transfer.obj
 0001:00006c88       ?CallCompletionRoutine@CUfnMddTransfer@@QAAXXZ 10007c88 f   usb_ufnmddbase_common_topaz_v1:transfer.obj
 0001:00006cc8       ?ReferenceTransferHandle@CUfnMddTransfer@@SAKPAV1@@Z 10007cc8 f   usb_ufnmddbase_common_topaz_v1:transfer.obj
 0001:00006d38       ?ConvertFromPddTransfer@CUfnMddTransfer@@SAPAV1@PAU_STransfer@@@Z 10007d38 f   usb_ufnmddbase_common_topaz_v1:transfer.obj
 0001:00006d40       ?DeRef@CRefObject@@QAAKXZ  10007d40 f i usb_ufnmddbase_common_topaz_v1:ufnbus.obj
 0001:00006d7c       ?IOControl@DefaultBusDriver@@UAAHKPAEK0KPAK@Z 10007d7c f i usb_ufnmddbase_common_topaz_v1:ufnbus.obj
 0001:00006db8       ??0CUfnBusDevice@@QAA@PBG000KPAX@Z 10007db8 f   usb_ufnmddbase_common_topaz_v1:ufnbus.obj
 0001:00006e2c       ?Init@DeviceFolder@@UAAHXZ 10007e2c f i usb_ufnmddbase_common_topaz_v1:ufnbus.obj
 0001:00006e40       ?SetPowerState@DeviceFolder@@UAAHW4_CEDEVICE_POWER_STATE@@@Z 10007e40 f i usb_ufnmddbase_common_topaz_v1:ufnbus.obj
 0001:00006e4c       ?GetPowerState@DeviceFolder@@UAA?AW4_CEDEVICE_POWER_STATE@@XZ 10007e4c f i usb_ufnmddbase_common_topaz_v1:ufnbus.obj
 0001:00006e54       ?Init@CUfnBusDevice@@UAAHXZ 10007e54 f i usb_ufnmddbase_common_topaz_v1:ufnbus.obj
 0001:00006e70       ??_GCUfnBusDevice@@UAAPAXI@Z 10007e70 f i usb_ufnmddbase_common_topaz_v1:ufnbus.obj
 0001:00006e70       ??_ECUfnBusDevice@@UAAPAXI@Z 10007e70 f i usb_ufnmddbase_common_topaz_v1:ufnbus.obj
 0001:00007040       ??0CUfnBus@@QAA@PBGPAUUFN_MDD_CONTEXT@@@Z 10008040 f   usb_ufnmddbase_common_topaz_v1:ufnbus.obj
 0001:00007078       ?PowerUp@DefaultBusDriver@@UAAHXZ 10008078 f i usb_ufnmddbase_common_topaz_v1:ufnbus.obj
 0001:00007080       ?PowerDown@DefaultBusDriver@@UAAHXZ 10008080 f i usb_ufnmddbase_common_topaz_v1:ufnbus.obj
 0001:00007088       ?Close@DefaultBusDriver@@UAAHXZ 10008088 f i usb_ufnmddbase_common_topaz_v1:ufnbus.obj
 0001:00007090       ?IsChildRemoved@DefaultBusDriver@@UAAHPBG@Z 10008090 f i usb_ufnmddbase_common_topaz_v1:ufnbus.obj
 0001:000070a0       ?Init@CUfnBus@@UAAHXZ      100080a0 f   usb_ufnmddbase_common_topaz_v1:ufnbus.obj
 0001:00007144       ?CreateChild@CUfnBus@@IAAKPBGPAPAVCUfnBusDevice@@@Z 10008144 f   usb_ufnmddbase_common_topaz_v1:ufnbus.obj
 0001:00007234       ?OpenFunctionKey@CUfnBus@@SAKPAPAUHKEY__@@K@Z 10008234 f   usb_ufnmddbase_common_topaz_v1:ufnbus.obj
 0001:00007264       ?TranslateChildBusAddr@CUfnBus@@UAAHPAU_CE_BUS_TRANSLATE_BUS_ADDR@@@Z 10008264 f   usb_ufnmddbase_common_topaz_v1:ufnbus.obj
 0001:000072f8       ?TranslateChildSystemAddr@CUfnBus@@UAAHPAU_CE_BUS_TRANSLATE_SYSTEM_ADDR@@@Z 100082f8 f   usb_ufnmddbase_common_topaz_v1:ufnbus.obj
 0001:0000738c       ?SetChildDevicePowerState@CUfnBus@@UAAHPAU_CE_BUS_POWER_STATE@@PAPAVDeviceFolder@@@Z 1000838c f   usb_ufnmddbase_common_topaz_v1:ufnbus.obj
 0001:00007434       ?GetChildDevicePowerState@CUfnBus@@UAAHPAU_CE_BUS_POWER_STATE@@PAPAVDeviceFolder@@@Z 10008434 f   usb_ufnmddbase_common_topaz_v1:ufnbus.obj
 0001:000074c4       ?SetChildDeviceConfigurationData@CUfnBus@@UAAHPAU_CE_BUS_DEVICE_CONFIGURATION_DATA@@PAPAVDeviceFolder@@@Z 100084c4 f   usb_ufnmddbase_common_topaz_v1:ufnbus.obj
 0001:00007554       ?GetChildDeviceConfigurationData@CUfnBus@@UAAHPAU_CE_BUS_DEVICE_CONFIGURATION_DATA@@PAPAVDeviceFolder@@@Z 10008554 f   usb_ufnmddbase_common_topaz_v1:ufnbus.obj
 0001:000075e4       ?GetBusNamePrefix@CUfnBus@@UAAKPAGK@Z 100085e4 f   usb_ufnmddbase_common_topaz_v1:ufnbus.obj
 0001:00007614       ?GetDefaultClientKey@CUfnBus@@QAAXPAGK@Z 10008614 f   usb_ufnmddbase_common_topaz_v1:ufnbus.obj
 0001:00007698       ?GetDefaultClientName@CUfnBus@@QAAKPAGK@Z 10008698 f   usb_ufnmddbase_common_topaz_v1:ufnbus.obj
 0001:00007778       ?PostInit@CUfnBus@@UAAHXZ  10008778 f   usb_ufnmddbase_common_topaz_v1:ufnbus.obj
 0001:00007880       ?IOControl@CUfnBus@@UAAHPAUUFN_MDD_BUS_OPEN_CONTEXT@@KPAEK1KPAK@Z 10008880 f   usb_ufnmddbase_common_topaz_v1:ufnbus.obj
 0001:00007ed8       ??0?$CFreePool@$03V?$fixed_block_allocator@$07@ce@@Utransfer_funcs@@@@QAA@I@Z 10008ed8 f i usb_ufnmddbase_common_topaz_v1:ufnbus.obj
 0001:00007f38       ??1?$CFreePool@$03V?$fixed_block_allocator@$07@ce@@Utransfer_funcs@@@@QAA@XZ 10008f38 f i usb_ufnmddbase_common_topaz_v1:ufnbus.obj
 0001:00008000       ?CleanUpAfterClient@CUfnBus@@IAAKXZ 10009000 f   usb_ufnmddbase_common_topaz_v1:ufnbus.obj
 0001:00008144       ?ActivateChild@CUfnBus@@UAAHPBG@Z 10009144 f   usb_ufnmddbase_common_topaz_v1:ufnbus.obj
 0001:0000822c       ?DeactivateChild@CUfnBus@@UAAHPBG@Z 1000922c f   usb_ufnmddbase_common_topaz_v1:ufnbus.obj
 0001:00008250       ??1CUfnBus@@UAA@XZ         10009250 f   usb_ufnmddbase_common_topaz_v1:ufnbus.obj
 0001:00008294       ??_ECUfnBus@@UAAPAXI@Z     10009294 f i usb_ufnmddbase_common_topaz_v1:ufnbus.obj
 0001:00008294       ??_GCUfnBus@@UAAPAXI@Z     10009294 f i usb_ufnmddbase_common_topaz_v1:ufnbus.obj
 0001:00008678       ?GetDefaultInterfaceCount@CConfiguration@@QBAKXZ 10009678 f i usb_ufnmddbase_common_topaz_v1:enum.obj
 0001:000086c0       ?SetInterface@CConfiguration@@QAAKKK@Z 100096c0 f i usb_ufnmddbase_common_topaz_v1:enum.obj
 0001:00008708       ?ResetInterfaces@CConfiguration@@QAAXXZ 10009708 f i usb_ufnmddbase_common_topaz_v1:enum.obj
 0001:00008748       ?SetConfiguration@CDevice@@QAAKK@Z 10009748 f i usb_ufnmddbase_common_topaz_v1:enum.obj
 0001:00008ea8       ?compact@?$CFreePool@$03V?$fixed_block_allocator@$07@ce@@Utransfer_funcs@@@@QAAXXZ 10009ea8 f i usb_ufnmddbase_common_topaz_v1:enum.obj
 0001:00008f64       ?UfnMdd_Notify@@YAHPAXKK@Z 10009f64 f   usb_ufnmddbase_common_topaz_v1:enum.obj
 0001:00009324       ?Prev@SVSTree@@QAAPAVSVSTNode@@PAV2@@Z 1000a324 f i ceosutil:utilmemf.obj
 0001:00009388       ?LocateLeftNeighbor@SVSTree@@QAAPAVSVSTNode@@K@Z 1000a388 f i ceosutil:utilmemf.obj
 0001:000093f4       svsutil_AllocFixedMemDescrSynch 1000a3f4 f   ceosutil:utilmemf.obj
 0001:0000945c       svsutil_GetFixed           1000a45c f   ceosutil:utilmemf.obj
 0001:00009530       svsutil_FreeFixed          1000a530 f   ceosutil:utilmemf.obj
 0001:0000956c       svsutil_ReleaseFixedNonEmpty 1000a56c f   ceosutil:utilmemf.obj
 0001:000095e0       svsutil_ReleaseFixedEmpty  1000a5e0 f   ceosutil:utilmemf.obj
 0001:00009618       ?DeleteSubtree@SVSTree@@IAAXPAVSVSTNode@@@Z 1000a618 f i ceosutil:utilmemf.obj
 0001:00009654       ??0SVSTree@@QAA@I@Z        1000a654 f i ceosutil:utilmemf.obj
 0001:000096f8       ?Next@SVSTree@@QAAPAVSVSTNode@@PAV2@@Z 1000a6f8 f i ceosutil:utilmemf.obj
 0001:0000975c       ?EnumStart@SVSTree@@UAAKXZ 1000a75c f i ceosutil:utilmemf.obj
 0001:00009794       ?EnumNext@SVSTree@@UAAKK@Z 1000a794 f i ceosutil:utilmemf.obj
 0001:00009798       ?EnumGetData@SVSTree@@UAAPAXK@Z 1000a798 f i ceosutil:utilmemf.obj
 0001:000097a0       ?EnumGetKey@SVSTree@@UAAKK@Z 1000a7a0 f i ceosutil:utilmemf.obj
 0001:000097a8       ?Empty@SVSTree@@QAAXXZ     1000a7a8 f i ceosutil:utilmemf.obj
 0001:000097f4       ??1SVSTree@@QAA@XZ         1000a7f4 f i ceosutil:utilmemf.obj
 0001:0000983c       ?SVSNewTree@@YAPAVSVSTree@@I@Z 1000a83c f i ceosutil:utilmemf.obj
 0001:000098c8       svsutil_CompactFixed       1000a8c8 f   ceosutil:utilmemf.obj
 0001:00009b48       svsutil_Initialize         1000ab48 f   ceosutil:utilmem.obj
 0001:00009b4c       svsutil_DeInitialize       1000ab4c f   ceosutil:utilmem.obj
 0001:00009b50       svsutil_Alloc              1000ab50 f   ceosutil:utilmem.obj
 0001:00009b54       svsutil_ReAlloc            1000ab54 f   ceosutil:utilmem.obj
 0001:00009b58       svsutil_Free               1000ab58 f   ceosutil:utilmem.obj
 0001:00009b5c       ?TreeInsert@SVSTree@@IAAXPAVSVSTNode@@@Z 1000ab5c f i ceosutil:utiltree.obj
 0001:00009bcc       ?LeftRotate@SVSTree@@IAAXPAVSVSTNode@@@Z 1000abcc f i ceosutil:utiltree.obj
 0001:00009c24       ?RightRotate@SVSTree@@IAAXPAVSVSTNode@@@Z 1000ac24 f i ceosutil:utiltree.obj
 0001:00009c7c       ?Insert@SVSTree@@QAAPAVSVSTNode@@KPAX@Z 1000ac7c f   ceosutil:utiltree.obj
 0001:00009dcc       ??_GCRefObject@@UAAPAXI@Z  1000adcc f i defbuslib:DefBus.obj
 0001:00009dcc       ??_ECRefObject@@UAAPAXI@Z  1000adcc f i defbuslib:DefBus.obj
 0001:00009df0       ??0CRegistryEdit@@QAA@PAUHKEY__@@PBG@Z 1000adf0 f i defbuslib:DefBus.obj
 0001:00009e3c       ?GetRegValue@CRegistryEdit@@QAAHPBGPAEK@Z 1000ae3c f i defbuslib:DefBus.obj
 0001:00009e8c       ?TranslateBusAddr@DefaultBusDriver@@QAAHW4_INTERFACE_TYPE@@KT_LARGE_INTEGER@@PAKPAT3@@Z 1000ae8c f i defbuslib:DefBus.obj
 0001:00009f08       ?TranslateSystemAddr@DefaultBusDriver@@QAAHW4_INTERFACE_TYPE@@KT_LARGE_INTEGER@@PAT3@@Z 1000af08 f i defbuslib:DefBus.obj
 0001:00009f7c       ?LoadDevice@DeviceFolder@@UAAHXZ 1000af7c f   defbuslib:DefBus.obj
 0001:0000a0f4       ?UnloadDevice@DeviceFolder@@UAAHXZ 1000b0f4 f   defbuslib:DefBus.obj
 0001:0000a128       ?EnableDevice@DeviceFolder@@UAAHK@Z 1000b128 f   defbuslib:DefBus.obj
 0001:0000a144       ?DisableDevice@DeviceFolder@@UAAHK@Z 1000b144 f   defbuslib:DefBus.obj
 0001:0000a160       ?IsDeviceDriverEnabled@DeviceFolder@@QAAHPAK@Z 1000b160 f   defbuslib:DefBus.obj
 0001:0000a1a0       ?SetConfigurationData@DeviceFolder@@UAAHPAU_CE_BUS_DEVICE_CONFIGURATION_DATA@@@Z 1000b1a0 f   defbuslib:DefBus.obj
 0001:0000a20c       ?GetConfigurationData@DeviceFolder@@UAAHPAU_CE_BUS_DEVICE_CONFIGURATION_DATA@@@Z 1000b20c f   defbuslib:DefBus.obj
 0001:0000a278       ??0DefaultBusDriver@@QAA@PBG@Z 1000b278 f   defbuslib:DefBus.obj
 0001:0000a2d0       ?PostInit@DefaultBusDriver@@UAAHXZ 1000b2d0 f i defbuslib:DefBus.obj
 0001:0000a2d8       ?Init@DefaultBusDriver@@UAAHXZ 1000b2d8 f   defbuslib:DefBus.obj
 0001:0000a2f4       ??1DefaultBusDriver@@UAA@XZ 1000b2f4 f   defbuslib:DefBus.obj
 0001:0000a394       ?TranslateChildBusAddr@DefaultBusDriver@@UAAHPAU_CE_BUS_TRANSLATE_BUS_ADDR@@@Z 1000b394 f   defbuslib:DefBus.obj
 0001:0000a3e0       ?TranslateChildSystemAddr@DefaultBusDriver@@UAAHPAU_CE_BUS_TRANSLATE_SYSTEM_ADDR@@@Z 1000b3e0 f   defbuslib:DefBus.obj
 0001:0000a424       ?SetChildDeviceConfigurationData@DefaultBusDriver@@UAAHPAU_CE_BUS_DEVICE_CONFIGURATION_DATA@@PAPAVDeviceFolder@@@Z 1000b424 f   defbuslib:DefBus.obj
 0001:0000a474       ?GetChildDeviceConfigurationData@DefaultBusDriver@@UAAHPAU_CE_BUS_DEVICE_CONFIGURATION_DATA@@PAPAVDeviceFolder@@@Z 1000b474 f   defbuslib:DefBus.obj
 0001:0000a4c4       ?SetChildDevicePowerState@DefaultBusDriver@@UAAHPAU_CE_BUS_POWER_STATE@@PAPAVDeviceFolder@@@Z 1000b4c4 f   defbuslib:DefBus.obj
 0001:0000a52c       ?GetChildDevicePowerState@DefaultBusDriver@@UAAHPAU_CE_BUS_POWER_STATE@@PAPAVDeviceFolder@@@Z 1000b52c f   defbuslib:DefBus.obj
 0001:0000a598       ?ActivateChild@DefaultBusDriver@@UAAHPBG@Z 1000b598 f   defbuslib:DefBus.obj
 0001:0000a5dc       ?DeactivateChild@DefaultBusDriver@@UAAHPBG@Z 1000b5dc f   defbuslib:DefBus.obj
 0001:0000a620       ?EnableChild@DefaultBusDriver@@UAAHPBGK@Z 1000b620 f   defbuslib:DefBus.obj
 0001:0000a66c       ?DisableChild@DefaultBusDriver@@UAAHPBGK@Z 1000b66c f   defbuslib:DefBus.obj
 0001:0000a6b8       ?IsChildEnabled@DefaultBusDriver@@QAAHPBGPAK@Z 1000b6b8 f   defbuslib:DefBus.obj
 0001:0000a714       ?GetBusNamePrefix@DefaultBusDriver@@UAAKPAGK@Z 1000b714 f   defbuslib:DefBus.obj
 0001:0000a76c       ?FastIOControl@DefaultBusDriver@@UAAHKPAEK0KPAKPAPAVDeviceFolder@@@Z 1000b76c f   defbuslib:DefBus.obj
 0001:0000ac00       ?GetChildByName@DefaultBusDriver@@UAAPAVDeviceFolder@@PBGPAPAV2@@Z 1000bc00 f   defbuslib:DefBus.obj
 0001:0000ad0c       ?InsertChild@DefaultBusDriver@@UAAHPAVDeviceFolder@@@Z 1000bd0c f   defbuslib:DefBus.obj
 0001:0000ad90       ?RemoveChildByName@DefaultBusDriver@@UAAHPBG@Z 1000bd90 f   defbuslib:DefBus.obj
 0001:0000ade4       ?RemoveChildByFolder@DefaultBusDriver@@UAAHPAVDeviceFolder@@@Z 1000bde4 f   defbuslib:DefBus.obj
 0001:0000ae7c       ?Open@DefaultBusDriver@@UAAHKK@Z 1000be7c f   defbuslib:DefBus.obj
 0001:0000ae8c       ??0DeviceFolder@@QAA@PBG0KKKKPAXK0@Z 1000be8c f   defbuslib:DefBus.obj
 0001:0000b13c       ??1DeviceFolder@@UAA@XZ    1000c13c f   defbuslib:DefBus.obj
 0001:0000b200       ??_GDefaultBusDriver@@UAAPAXI@Z 1000c200 f i defbuslib:DefBus.obj
 0001:0000b200       ??_EDefaultBusDriver@@UAAPAXI@Z 1000c200 f i defbuslib:DefBus.obj
 0001:0000b224       ??_GDeviceFolder@@UAAPAXI@Z 1000c224 f i defbuslib:DefBus.obj
 0001:0000b224       ??_EDeviceFolder@@UAAPAXI@Z 1000c224 f i defbuslib:DefBus.obj
 0001:0000b248       BusChildIoControl          1000c248 f   ceddk:CEDDK.dll
 0001:0000b258       CloseBusAccessHandle       1000c258 f   ceddk:CEDDK.dll
 0001:0000b268       CreateBusAccessHandle      1000c268 f   ceddk:CEDDK.dll
 0001:0000b278       HalTranslateBusAddress     1000c278 f   ceddk:CEDDK.dll
 0001:0000b288       TranslateBusAddr           1000c288 f   ceddk:CEDDK.dll
 0001:0000b298       HalTranslateSystemAddress  1000c298 f   ceddk:CEDDK.dll
 0001:0000b2a8       TranslateSystemAddr        1000c2a8 f   ceddk:CEDDK.dll
 0001:0000b2b8       HalSetBusDataByOffset      1000c2b8 f   ceddk:CEDDK.dll
 0001:0000b2c8       HalGetBusDataByOffset      1000c2c8 f   ceddk:CEDDK.dll
 0001:0000b2d8       Sleep                      1000c2d8 f   coredll:COREDLL.dll
 0001:0000b2e8       InterlockedCompareExchange 1000c2e8 f   coredll:COREDLL.dll
 0001:0000b2f8       GetLastError               1000c2f8 f   coredll:COREDLL.dll
 0001:0000b308       MapViewOfFile              1000c308 f   coredll:COREDLL.dll
 0001:0000b318       CreateFileMappingW         1000c318 f   coredll:COREDLL.dll
 0001:0000b328       CloseHandle                1000c328 f   coredll:COREDLL.dll
 0001:0000b338       UnmapViewOfFile            1000c338 f   coredll:COREDLL.dll
 0001:0000b348       KernelIoControl            1000c348 f   coredll:COREDLL.dll
 0001:0000b358       InitializeCriticalSection  1000c358 f   coredll:COREDLL.dll
 0001:0000b368       DeleteCriticalSection      1000c368 f   coredll:COREDLL.dll
 0001:0000b378       EnterCriticalSection       1000c378 f   coredll:COREDLL.dll
 0001:0000b388       LeaveCriticalSection       1000c388 f   coredll:COREDLL.dll
 0001:0000b398       LocalFree                  1000c398 f   coredll:COREDLL.dll
 0001:0000b3a8       RegCloseKey                1000c3a8 f   coredll:COREDLL.dll
 0001:0000b3b8       SetLastError               1000c3b8 f   coredll:COREDLL.dll
 0001:0000b3c8       RegOpenKeyExW              1000c3c8 f   coredll:COREDLL.dll
 0001:0000b3d8       DisableThreadLibraryCalls  1000c3d8 f   coredll:COREDLL.dll
 0001:0000b3e8       LocalAlloc                 1000c3e8 f   coredll:COREDLL.dll
 0001:0000b3f8       OpenDeviceKey              1000c3f8 f   coredll:COREDLL.dll
 0001:0000b408       CreateEventW               1000c408 f   coredll:COREDLL.dll
 0001:0000b418       InterlockedExchange        1000c418 f   coredll:COREDLL.dll
 0001:0000b428       StringCchCopyW             1000c428 f   coredll:COREDLL.dll
 0001:0000b438       InterlockedIncrement       1000c438 f   coredll:COREDLL.dll
 0001:0000b448       InterlockedDecrement       1000c448 f   coredll:COREDLL.dll
 0001:0000b458       EventModify                1000c458 f   coredll:COREDLL.dll
 0001:0000b468       RegQueryValueExW           1000c468 f   coredll:COREDLL.dll
 0001:0000b478       StringCchPrintfW           1000c478 f   coredll:COREDLL.dll
 0001:0000b488       GetDeviceInformationByDeviceHandle 1000c488 f   coredll:COREDLL.dll
 0001:0000b498       RegSetValueExW             1000c498 f   coredll:COREDLL.dll
 0001:0000b4a8       LoadLibraryW               1000c4a8 f   coredll:COREDLL.dll
 0001:0000b4b8       RegEnumKeyExW              1000c4b8 f   coredll:COREDLL.dll
 0001:0000b4c8       WaitForSingleObject        1000c4c8 f   coredll:COREDLL.dll
 0001:0000b4d8       ActivateDeviceEx           1000c4d8 f   coredll:COREDLL.dll
 0001:0000b4e8       FreeLibrary                1000c4e8 f   coredll:COREDLL.dll
 0001:0000b4f8       GetProcAddressW            1000c4f8 f   coredll:COREDLL.dll
 0001:0000b508       LoadDriver                 1000c508 f   coredll:COREDLL.dll
 0001:0000b518       DeactivateDevice           1000c518 f   coredll:COREDLL.dll
 0001:0000b528       EnableDeviceDriver         1000c528 f   coredll:COREDLL.dll
 0001:0000b538       DisableDeviceDriver        1000c538 f   coredll:COREDLL.dll
 0001:0000b548       GetDeviceDriverStatus      1000c548 f   coredll:COREDLL.dll
 0001:0000b558       GetDeviceHandleFromContext 1000c558 f   coredll:COREDLL.dll
 0001:0000b568       DDKClockSetGatingMode      1000c568 f   cspddk:CSPDDK.dll
 0001:0000b578       DDKClockGetGatingMode      1000c578 f   cspddk:CSPDDK.dll
 0001:0000b588       DDKClockConfigBaud         1000c588 f   cspddk:CSPDDK.dll
 0001:0000b598       _DllEntryCRTStartup        1000c598 f   corelib0:pegdentry.obj
 0001:0000b5dc       _onexit                    1000c5dc f   corelib0:onexit.obj
 0001:0000b6ac       atexit                     1000c6ac f   corelib0:onexit.obj
 0001:0000b6c4       __GSHandlerCheckCommon     1000c6c4 f   corelib0:gshandler.obj
 0001:0000b6fc       __GSHandlerCheck           1000c6fc f   corelib0:gshandler.obj
 0001:0000b71c       __security_init_cookie     1000c71c f   corelib0:seccinit.obj
 0001:0000b768       __security_check_cookie    1000c768 f   corelib0:armsecgs.obj
 0001:0000b778       __gsfailure                1000c778     corelib0:armsecgs.obj
 0001:0000b87c       _cexit                     1000c87c f   corelib0:cexit.obj
 0001:0000b88c       _initterm                  1000c88c f   corelib0:crt0dat.obj
 0001:0000b8b8       _cinit                     1000c8b8 f   corelib0:crt0dat.obj
 0001:0000b918       __crt_ExitProcess          1000c918 f   corelib0:exitproc_proxy.obj
 0001:0000b924       ??2@YAPAXI@Z               1000c924 f   corelib1:COREDLL.dll
 0001:0000b934       ??3@YAXPAX@Z               1000c934 f   corelib1:COREDLL.dll
 0001:0000b944       __C_specific_handler       1000c944 f   corelib1:COREDLL.dll
 0001:0000b954       _purecall                  1000c954 f   corelib1:COREDLL.dll
 0001:0000b964       memcpy                     1000c964 f   corelib1:COREDLL.dll
 0001:0000b974       wcslen                     1000c974 f   corelib1:COREDLL.dll
 0001:0000b984       memset                     1000c984 f   corelib1:COREDLL.dll
 0001:0000b994       ??_V@YAXPAX@Z              1000c994 f   corelib1:COREDLL.dll
 0001:0000b9a4       ??_U@YAPAXI@Z              1000c9a4 f   corelib1:COREDLL.dll
 0001:0000b9b4       malloc                     1000c9b4 f   corelib1:COREDLL.dll
 0001:0000b9c4       realloc                    1000c9c4 f   corelib1:COREDLL.dll
 0001:0000b9d4       free                       1000c9d4 f   corelib1:COREDLL.dll
 0001:0000b9e4       _wcsicmp                   1000c9e4 f   corelib1:COREDLL.dll
 0001:0000b9f4       _wcsnicmp                  1000c9f4 f   corelib1:COREDLL.dll
 0001:0000ba04       _wcsdup                    1000ca04 f   corelib1:COREDLL.dll
 0001:0000ba14       _msize                     1000ca14 f   corelib1:COREDLL.dll
 0001:0000ba24       __security_gen_cookie2     1000ca24 f   corelib1:COREDLL.dll
 0001:0000ba34       __report_gsfailure         1000ca34 f   corelib1:COREDLL.dll
 0001:0000baf0       ClearUsbstsUI              1000caf0 f   usb_usbfn_mx25_topaz_v1:i_pdd.obj
 0001:0000c26c       UfnPdd_PowerDown           1000d26c f   usb_usbfn_mx25_topaz_v1:i_pdd.obj
 0001:0000c350       UfnPdd_PowerUp             1000d350 f   usb_usbfn_mx25_topaz_v1:i_pdd.obj
 0001:0000c43c       UpdateDevicePower          1000d43c f   usb_usbfn_mx25_topaz_v1:i_pdd.obj
 0001:0000c4f4       SetupEvent                 1000d4f4 f   usb_usbfn_mx25_topaz_v1:i_pdd.obj
 0001:0000c630       CopyFromUncachedBuffer     1000d630 f   usb_usbfn_mx25_topaz_v1:i_pdd.obj
 0001:0000c9ec       UfnPdd_IssueTransfer       1000d9ec f   usb_usbfn_mx25_topaz_v1:i_pdd.obj
 0001:0000cfc0       UfnPdd_AbortTransfer       1000dfc0 f   usb_usbfn_mx25_topaz_v1:i_pdd.obj
 0001:0000d168       UfnPdd_StallEndpoint       1000e168 f   usb_usbfn_mx25_topaz_v1:i_pdd.obj
 0001:0000d1f4       UfnPdd_ClearEndpointStall  1000e1f4 f   usb_usbfn_mx25_topaz_v1:i_pdd.obj
 0001:0000d294       UfnPdd_IsEndpointHalted    1000e294 f   usb_usbfn_mx25_topaz_v1:i_pdd.obj
 0001:0000d2fc       UfnPdd_SendControlStatusHandshake 1000e2fc f   usb_usbfn_mx25_topaz_v1:i_pdd.obj
 0001:0000d37c       UfnPdd_InitiateRemoteWakeup 1000e37c f   usb_usbfn_mx25_topaz_v1:i_pdd.obj
 0001:0000d384       SetPowerState              1000e384 f   usb_usbfn_mx25_topaz_v1:i_pdd.obj
 0001:0000d3c8       UfnPdd_IOControl           1000e3c8 f   usb_usbfn_mx25_topaz_v1:i_pdd.obj
 0001:0000d5d8       UfnPdd_Deinit              1000e5d8 f   usb_usbfn_mx25_topaz_v1:i_pdd.obj
 0001:0000d5e8       UfnPdd_DeregisterDevice    1000e5e8 f   usb_usbfn_mx25_topaz_v1:i_pdd.obj
 0001:0000d5f0       UfnPdd_Stop                1000e5f0 f   usb_usbfn_mx25_topaz_v1:i_pdd.obj
 0001:0000d65c       UfnPdd_DeinitEndpoint      1000e65c f   usb_usbfn_mx25_topaz_v1:i_pdd.obj
 0001:0000d700       UfnPdd_InitEndpoint        1000e700 f   usb_usbfn_mx25_topaz_v1:i_pdd.obj
 0001:0000d81c       UfnPdd_SetAddress          1000e81c f   usb_usbfn_mx25_topaz_v1:i_pdd.obj
 0001:0000d850       UfnPdd_Start               1000e850 f   usb_usbfn_mx25_topaz_v1:i_pdd.obj
 0001:0000d940       UfnPdd_RegisterDevice      1000e940 f   usb_usbfn_mx25_topaz_v1:i_pdd.obj
 0001:0000db6c       UfnPdd_IsEndpointSupportable 1000eb6c f   usb_usbfn_mx25_topaz_v1:i_pdd.obj
 0001:0000db88       UfnPdd_IsConfigurationSupportable 1000eb88 f   usb_usbfn_mx25_topaz_v1:i_pdd.obj
 0001:0000dcdc       UfnPdd_Init                1000ecdc f   usb_usbfn_mx25_topaz_v1:i_pdd.obj
 0001:0000dfd8       UfnPdd_DllEntry            1000efd8 f   usb_usbfn_mx25_topaz_v1:i_pdd.obj
 0001:0000dfe0       CheckEndpoint              1000efe0 f   usb_usbfn_mx25_topaz_v1:i_pdd.obj
 0001:0000e464       InterruptHandle            1000f464 f   usb_usbfn_mx25_topaz_v1:i_pdd.obj
 0001:0000ea5c       FslUfnIsUSBKitlEnable      1000fa5c f   usb_usbfn_os_mx25_topaz_v1:i_os.obj
 0001:0000eac8       FslUfnGetUsbFnPdd          1000fac8 f   usb_usbfn_os_mx25_topaz_v1:i_os.obj
 0001:0000ead8       FslUfnRequestIrq           1000fad8 f   usb_usbfn_os_mx25_topaz_v1:i_os.obj
 0001:0000eb70       FslUfnGetDMABuffer         1000fb70 f   usb_usbfn_os_mx25_topaz_v1:i_os.obj
 0001:0000ec20       FslUfnTrigIrq              1000fc20 f   usb_usbfn_os_mx25_topaz_v1:i_os.obj
 0001:0000ec2c       FslUfnDeinit               1000fc2c f   usb_usbfn_os_mx25_topaz_v1:i_os.obj
 0001:0000ed88       InterruptThread            1000fd88 f   usb_usbfn_os_mx25_topaz_v1:i_os.obj
 0001:0000efc8       FslUfnGetPageNumber        1000ffc8 f   usb_usbfn_os_mx25_topaz_v1:i_os.obj
 0001:0000efe8       FslUfnGetPageSize          1000ffe8 f   usb_usbfn_os_mx25_topaz_v1:i_os.obj
 0001:0000eff8       FslUfnGetPageShift         1000fff8 f   usb_usbfn_os_mx25_topaz_v1:i_os.obj
 0001:0000f008       FslInitializeCriticalSection 10010008 f   usb_usbfn_os_mx25_topaz_v1:i_os.obj
 0001:0000f00c       FslEnterCriticalSection    1001000c f   usb_usbfn_os_mx25_topaz_v1:i_os.obj
 0001:0000f010       FslLeaveCriticalSection    10010010 f   usb_usbfn_os_mx25_topaz_v1:i_os.obj
 0001:0000f014       FslUfnCreateThread         10010014 f   usb_usbfn_os_mx25_topaz_v1:i_os.obj
 0001:0000f47c       GetDeviceRegistryParams    1001047c f   usb_usbfn_os_mx25_topaz_v1:i_registry.obj
 0001:0000f618       SetDevicePowerState        10010618 f   ceddk:CEDDK.dll
 0001:0000f628       MmMapIoSpace               10010628 f   ceddk:CEDDK.dll
 0001:0000f638       HalAllocateCommonBuffer    10010638 f   ceddk:CEDDK.dll
 0001:0000f648       HalFreeCommonBuffer        10010648 f   ceddk:CEDDK.dll
 0001:0000f658       MmUnmapIoSpace             10010658 f   ceddk:CEDDK.dll
 0001:0000f668       TerminateProcess           10010668 f   coredll:COREDLL.dll
 0001:0000f678       CeLogData                  10010678 f   coredll:COREDLL.dll
 0001:0000f688       StringCchLengthW           10010688 f   coredll:COREDLL.dll
 0001:0000f698       StringCchVPrintfW          10010698 f   coredll:COREDLL.dll
 0001:0000f6a8       SetInterruptEvent          100106a8 f   coredll:COREDLL.dll
 0001:0000f6b8       UnlockPages                100106b8 f   coredll:COREDLL.dll
 0001:0000f6c8       CacheSync                  100106c8 f   coredll:COREDLL.dll
 0001:0000f6d8       CeCloseCallerBuffer        100106d8 f   coredll:COREDLL.dll
 0001:0000f6e8       LockPages                  100106e8 f   coredll:COREDLL.dll
 0001:0000f6f8       CeOpenCallerBuffer         100106f8 f   coredll:COREDLL.dll
 0001:0000f708       InterruptDisable           10010708 f   coredll:COREDLL.dll
 0001:0000f718       CacheRangeFlush            10010718 f   coredll:COREDLL.dll
 0001:0000f728       InterruptInitialize        10010728 f   coredll:COREDLL.dll
 0001:0000f738       AllocPhysMem               10010738 f   coredll:COREDLL.dll
 0001:0000f748       FreePhysMem                10010748 f   coredll:COREDLL.dll
 0001:0000f758       ExitThread                 10010758 f   coredll:COREDLL.dll
 0001:0000f768       InterruptDone              10010768 f   coredll:COREDLL.dll
 0001:0000f778       StringCchCatW              10010778 f   coredll:COREDLL.dll
 0001:0000f788       CeSetThreadPriority        10010788 f   coredll:COREDLL.dll
 0001:0000f798       CreateThread               10010798 f   coredll:COREDLL.dll
 0001:0000f7a8       wcstoul                    100107a8 f   corelib1:COREDLL.dll
 0001:0000f7bc       ??__Fcs@?1??get_lock@?$singleton@V?$free_list@$0GE@Vallocator@ce@@@ce@@$03V?$static_allocator@V?$free_list@$0GE@Vallocator@ce@@@ce@@$03@2@@ce@@KAAAVcritical_section@2@XZ@YAXXZ 100107bc f i usb_ufnmddbase_common_topaz_v1:ufnmdd.obj
 0001:0000f8d0       __IMPORT_DESCRIPTOR_CEDDK  100108d0     ceddk:CEDDK.dll
 0001:0000f8e4       __IMPORT_DESCRIPTOR_COREDLL 100108e4     coredll:COREDLL.dll
 0001:0000f8f8       __IMPORT_DESCRIPTOR_CSPDDK 100108f8     cspddk:CSPDDK.dll
 0001:0000f90c       __NULL_IMPORT_DESCRIPTOR   1001090c     ceddk:CEDDK.dll
 0002:00000000       __imp_BusChildIoControl    10011000     ceddk:CEDDK.dll
 0002:00000004       __imp_CloseBusAccessHandle 10011004     ceddk:CEDDK.dll
 0002:00000008       __imp_CreateBusAccessHandle 10011008     ceddk:CEDDK.dll
 0002:0000000c       __imp_HalTranslateBusAddress 1001100c     ceddk:CEDDK.dll
 0002:00000010       __imp_TranslateBusAddr     10011010     ceddk:CEDDK.dll
 0002:00000014       __imp_HalTranslateSystemAddress 10011014     ceddk:CEDDK.dll
 0002:00000018       __imp_TranslateSystemAddr  10011018     ceddk:CEDDK.dll
 0002:0000001c       __imp_HalSetBusDataByOffset 1001101c     ceddk:CEDDK.dll
 0002:00000020       __imp_HalGetBusDataByOffset 10011020     ceddk:CEDDK.dll
 0002:00000024       __imp_HalFreeCommonBuffer  10011024     ceddk:CEDDK.dll
 0002:00000028       __imp_HalAllocateCommonBuffer 10011028     ceddk:CEDDK.dll
 0002:0000002c       __imp_MmMapIoSpace         1001102c     ceddk:CEDDK.dll
 0002:00000030       __imp_SetDevicePowerState  10011030     ceddk:CEDDK.dll
 0002:00000034       __imp_MmUnmapIoSpace       10011034     ceddk:CEDDK.dll
 0002:00000038       \177CEDDK_NULL_THUNK_DATA  10011038     ceddk:CEDDK.dll
 0002:0000003c       __imp_CloseHandle          1001103c     coredll:COREDLL.dll
 0002:00000040       __imp_UnmapViewOfFile      10011040     coredll:COREDLL.dll
 0002:00000044       __imp_KernelIoControl      10011044     coredll:COREDLL.dll
 0002:00000048       __imp_InitializeCriticalSection 10011048     coredll:COREDLL.dll
 0002:0000004c       __imp_DeleteCriticalSection 1001104c     coredll:COREDLL.dll
 0002:00000050       __imp_EnterCriticalSection 10011050     coredll:COREDLL.dll
 0002:00000054       __imp_LeaveCriticalSection 10011054     coredll:COREDLL.dll
 0002:00000058       __imp_LocalFree            10011058     coredll:COREDLL.dll
 0002:0000005c       __imp_RegCloseKey          1001105c     coredll:COREDLL.dll
 0002:00000060       __imp_SetLastError         10011060     coredll:COREDLL.dll
 0002:00000064       __imp_RegOpenKeyExW        10011064     coredll:COREDLL.dll
 0002:00000068       __imp_DisableThreadLibraryCalls 10011068     coredll:COREDLL.dll
 0002:0000006c       __imp_LocalAlloc           1001106c     coredll:COREDLL.dll
 0002:00000070       __imp_OpenDeviceKey        10011070     coredll:COREDLL.dll
 0002:00000074       __imp_CreateEventW         10011074     coredll:COREDLL.dll
 0002:00000078       __imp_InterlockedExchange  10011078     coredll:COREDLL.dll
 0002:0000007c       __imp_StringCchCopyW       1001107c     coredll:COREDLL.dll
 0002:00000080       __imp_InterlockedIncrement 10011080     coredll:COREDLL.dll
 0002:00000084       __imp_InterlockedDecrement 10011084     coredll:COREDLL.dll
 0002:00000088       __imp_EventModify          10011088     coredll:COREDLL.dll
 0002:0000008c       __imp_RegQueryValueExW     1001108c     coredll:COREDLL.dll
 0002:00000090       __imp_StringCchPrintfW     10011090     coredll:COREDLL.dll
 0002:00000094       __imp_GetDeviceInformationByDeviceHandle 10011094     coredll:COREDLL.dll
 0002:00000098       __imp_RegSetValueExW       10011098     coredll:COREDLL.dll
 0002:0000009c       __imp_CreateFileMappingW   1001109c     coredll:COREDLL.dll
 0002:000000a0       __imp_RegEnumKeyExW        100110a0     coredll:COREDLL.dll
 0002:000000a4       __imp_WaitForSingleObject  100110a4     coredll:COREDLL.dll
 0002:000000a8       __imp_ActivateDeviceEx     100110a8     coredll:COREDLL.dll
 0002:000000ac       __imp_FreeLibrary          100110ac     coredll:COREDLL.dll
 0002:000000b0       __imp_GetProcAddressW      100110b0     coredll:COREDLL.dll
 0002:000000b4       __imp_LoadDriver           100110b4     coredll:COREDLL.dll
 0002:000000b8       __imp_DeactivateDevice     100110b8     coredll:COREDLL.dll
 0002:000000bc       __imp_EnableDeviceDriver   100110bc     coredll:COREDLL.dll
 0002:000000c0       __imp_DisableDeviceDriver  100110c0     coredll:COREDLL.dll
 0002:000000c4       __imp_GetDeviceDriverStatus 100110c4     coredll:COREDLL.dll
 0002:000000c8       __imp_GetDeviceHandleFromContext 100110c8     coredll:COREDLL.dll
 0002:000000cc       __imp_CreateThread         100110cc     coredll:COREDLL.dll
 0002:000000d0       __imp_CeSetThreadPriority  100110d0     coredll:COREDLL.dll
 0002:000000d4       __imp_StringCchCatW        100110d4     coredll:COREDLL.dll
 0002:000000d8       __imp_??2@YAPAXI@Z         100110d8     corelib1:COREDLL.dll
 0002:000000dc       __imp_??3@YAXPAX@Z         100110dc     corelib1:COREDLL.dll
 0002:000000e0       __imp___C_specific_handler 100110e0     corelib1:COREDLL.dll
 0002:000000e4       __imp__purecall            100110e4     corelib1:COREDLL.dll
 0002:000000e8       __imp_memcpy               100110e8     corelib1:COREDLL.dll
 0002:000000ec       __imp_wcslen               100110ec     corelib1:COREDLL.dll
 0002:000000f0       __imp_memset               100110f0     corelib1:COREDLL.dll
 0002:000000f4       __imp_??_V@YAXPAX@Z        100110f4     corelib1:COREDLL.dll
 0002:000000f8       __imp_??_U@YAPAXI@Z        100110f8     corelib1:COREDLL.dll
 0002:000000fc       __imp_malloc               100110fc     corelib1:COREDLL.dll
 0002:00000100       __imp_realloc              10011100     corelib1:COREDLL.dll
 0002:00000104       __imp_free                 10011104     corelib1:COREDLL.dll
 0002:00000108       __imp__wcsicmp             10011108     corelib1:COREDLL.dll
 0002:0000010c       __imp__wcsnicmp            1001110c     corelib1:COREDLL.dll
 0002:00000110       __imp__wcsdup              10011110     corelib1:COREDLL.dll
 0002:00000114       __imp__msize               10011114     corelib1:COREDLL.dll
 0002:00000118       __imp___security_gen_cookie2 10011118     corelib1:COREDLL.dll
 0002:0000011c       __imp___report_gsfailure   1001111c     corelib1:COREDLL.dll
 0002:00000120       __imp_MapViewOfFile        10011120     coredll:COREDLL.dll
 0002:00000124       __imp_GetLastError         10011124     coredll:COREDLL.dll
 0002:00000128       __imp_InterlockedCompareExchange 10011128     coredll:COREDLL.dll
 0002:0000012c       __imp_Sleep                1001112c     coredll:COREDLL.dll
 0002:00000130       __imp_LoadLibraryW         10011130     coredll:COREDLL.dll
 0002:00000134       __imp_TerminateProcess     10011134     coredll:COREDLL.dll
 0002:00000138       __imp_CeLogData            10011138     coredll:COREDLL.dll
 0002:0000013c       __imp_StringCchLengthW     1001113c     coredll:COREDLL.dll
 0002:00000140       __imp_StringCchVPrintfW    10011140     coredll:COREDLL.dll
 0002:00000144       __imp_SetInterruptEvent    10011144     coredll:COREDLL.dll
 0002:00000148       __imp_UnlockPages          10011148     coredll:COREDLL.dll
 0002:0000014c       __imp_CacheSync            1001114c     coredll:COREDLL.dll
 0002:00000150       __imp_CeCloseCallerBuffer  10011150     coredll:COREDLL.dll
 0002:00000154       __imp_LockPages            10011154     coredll:COREDLL.dll
 0002:00000158       __imp_CeOpenCallerBuffer   10011158     coredll:COREDLL.dll
 0002:0000015c       __imp_InterruptDisable     1001115c     coredll:COREDLL.dll
 0002:00000160       __imp_CacheRangeFlush      10011160     coredll:COREDLL.dll
 0002:00000164       __imp_InterruptInitialize  10011164     coredll:COREDLL.dll
 0002:00000168       __imp_AllocPhysMem         10011168     coredll:COREDLL.dll
 0002:0000016c       __imp_FreePhysMem          1001116c     coredll:COREDLL.dll
 0002:00000170       __imp_ExitThread           10011170     coredll:COREDLL.dll
 0002:00000174       __imp_InterruptDone        10011174     coredll:COREDLL.dll
 0002:00000178       __imp_wcstoul              10011178     corelib1:COREDLL.dll
 0002:0000017c       \177COREDLL_NULL_THUNK_DATA 1001117c     coredll:COREDLL.dll
 0002:00000180       __imp_DDKClockGetGatingMode 10011180     cspddk:CSPDDK.dll
 0002:00000184       __imp_DDKClockSetGatingMode 10011184     cspddk:CSPDDK.dll
 0002:00000188       __imp_DDKClockConfigBaud   10011188     cspddk:CSPDDK.dll
 0002:0000018c       \177CSPDDK_NULL_THUNK_DATA 1001118c     cspddk:CSPDDK.dll
 0002:00000190       g_funcAlloc                10011190     ceosutil:utilmem.obj
 0002:00000194       g_funcFree                 10011194     ceosutil:utilmem.obj
 0002:00000198       g_funcRealloc              10011198     ceosutil:utilmem.obj
 0002:0000019c       __security_cookie          1001119c     corelib0:seccinit.obj
 0002:000001a0       __security_cookie_complement 100111a0     corelib0:seccinit.obj
 0002:000001c0       m_hUSBClockGatingHandle    100111c0     i_usbclock.obj
 0002:000001c4       pUSBClkGating              100111c4     i_usbclock.obj
 0002:000001d0       ?s_rgbBuffer@?$CTransferQueue@VCUfnMddTransfer@@@@0PAEA 100111d0     usb_ufnmddbase_common_topaz_v1:ufnmdd.obj
 0002:000001ec       ?s_pListStructAllocator@?$CTransferQueue@VCUfnMddTransfer@@@@0PAV?$fixed_block_allocator@$0BE@@ce@@A 100111ec     usb_ufnmddbase_common_topaz_v1:ufnmdd.obj
 0002:000001f0       ??_B?1??get_lock@?$singleton@V?$free_list@$0GE@Vallocator@ce@@@ce@@$03V?$static_allocator@V?$free_list@$0GE@Vallocator@ce@@@ce@@$03@2@@ce@@KAAAVcritical_section@2@XZ@51 100111f0     usb_ufnmddbase_common_topaz_v1:ufnmdd.obj
 0002:000001f4       ?cs@?1??get_lock@?$singleton@V?$free_list@$0GE@Vallocator@ce@@@ce@@$03V?$static_allocator@V?$free_list@$0GE@Vallocator@ce@@@ce@@$03@2@@ce@@KAAAVcritical_section@3@XZ@4V43@A 100111f4     usb_ufnmddbase_common_topaz_v1:ufnmdd.obj
 0002:00000208       ?_factory@?$singleton@V?$free_list@$0GE@Vallocator@ce@@@ce@@$03V?$static_allocator@V?$free_list@$0GE@Vallocator@ce@@@ce@@$03@2@@ce@@1Ulock_factory@12@A 10011208     usb_ufnmddbase_common_topaz_v1:ufnmdd.obj
 0002:0000020c       g_pvAllocData              1001120c     ceosutil:utilmem.obj
 0002:00000210       g_pvFreeData               10011210     ceosutil:utilmem.obj
 0002:00000214       _exitflag                  10011214     corelib0:cexit.obj
 0002:00000220       g_csRegister               10011220     <common>
 0002:00000234       __onexitend                10011234     <common>
 0002:00000238       __onexitbegin              10011238     <common>

 entry point at        0001:0000b598

 Static symbols

 0001:0000067c       InitializeMux              1000167c f   hwinit.obj
 0001:000006a0       SelectUSBCore              100016a0 f   hwinit.obj
 0001:000006cc       InitializeTransceiver      100016cc f   hwinit.obj
 0001:000017e0       ?IsPddInterfaceInfoValid@@YAHPAU_UFN_PDD_INTERFACE_INFO@@@Z 100027e0 f   usb_ufnmddbase_common_topaz_v1:ufnmdd.obj
 0001:00002470       ?FreeContext@@YAXPAUUFN_MDD_CONTEXT@@@Z 10003470 f   usb_ufnmddbase_common_topaz_v1:ufnmdd.obj
 0001:00004f98       ?FillBuffer@@YAKPAPAEPAKPBXK@Z 10005f98 f   usb_ufnmddbase_common_topaz_v1:descript.obj
 0001:00006ea0       ?GetUfnDescription@@YAHPAUHKEY__@@PAGK@Z 10007ea0 f   usb_ufnmddbase_common_topaz_v1:ufnbus.obj
 0001:00006f08       ?AllocEndpoints@@YAKPAUUFN_MDD_CONTEXT@@@Z 10007f08 f   usb_ufnmddbase_common_topaz_v1:ufnbus.obj
 0001:000082b8       ?EnumTransferComplete@@YAKPAX@Z 100092b8 f   usb_ufnmddbase_common_topaz_v1:enum.obj
 0001:0000830c       ?SetupTx@@YAXPAUUFN_MDD_CONTEXT@@PAXKK@Z 1000930c f   usb_ufnmddbase_common_topaz_v1:enum.obj
 0001:00008368       ?ProcessGetDescriptor@@YA?AW4CONTROL_RESPONSE@@PAUUFN_MDD_CONTEXT@@U_USB_DEVICE_REQUEST@@K@Z 10009368 f   usb_ufnmddbase_common_topaz_v1:enum.obj
 0001:000083ec       ?ProcessSetDescriptor@@YA?AW4CONTROL_RESPONSE@@PAUUFN_MDD_CONTEXT@@U_USB_DEVICE_REQUEST@@K@Z 100093ec f   usb_ufnmddbase_common_topaz_v1:enum.obj
 0001:00008400       ?ProcessSetAddress@@YA?AW4CONTROL_RESPONSE@@PAUUFN_MDD_CONTEXT@@U_USB_DEVICE_REQUEST@@K@Z 10009400 f   usb_ufnmddbase_common_topaz_v1:enum.obj
 0001:0000848c       ?ProcessClearFeature@@YA?AW4CONTROL_RESPONSE@@PAUUFN_MDD_CONTEXT@@U_USB_DEVICE_REQUEST@@K@Z 1000948c f   usb_ufnmddbase_common_topaz_v1:enum.obj
 0001:00008554       ?ProcessSetFeature@@YA?AW4CONTROL_RESPONSE@@PAUUFN_MDD_CONTEXT@@U_USB_DEVICE_REQUEST@@K@Z 10009554 f   usb_ufnmddbase_common_topaz_v1:enum.obj
 0001:00008664       ?ProcessSyncFrame@@YA?AW4CONTROL_RESPONSE@@PAUUFN_MDD_CONTEXT@@U_USB_DEVICE_REQUEST@@K@Z 10009664 f   usb_ufnmddbase_common_topaz_v1:enum.obj
 0001:00008794       ?ProcessGetConfiguration@@YA?AW4CONTROL_RESPONSE@@PAUUFN_MDD_CONTEXT@@U_USB_DEVICE_REQUEST@@K@Z 10009794 f   usb_ufnmddbase_common_topaz_v1:enum.obj
 0001:000087dc       ?ProcessGetInterface@@YA?AW4CONTROL_RESPONSE@@PAUUFN_MDD_CONTEXT@@U_USB_DEVICE_REQUEST@@K@Z 100097dc f   usb_ufnmddbase_common_topaz_v1:enum.obj
 0001:00008854       ?ProcessGetStatus@@YA?AW4CONTROL_RESPONSE@@PAUUFN_MDD_CONTEXT@@U_USB_DEVICE_REQUEST@@K@Z 10009854 f   usb_ufnmddbase_common_topaz_v1:enum.obj
 0001:000089c4       ?ProcessSetConfiguration@@YA?AW4CONTROL_RESPONSE@@PAUUFN_MDD_CONTEXT@@U_USB_DEVICE_REQUEST@@K@Z 100099c4 f   usb_ufnmddbase_common_topaz_v1:enum.obj
 0001:00008bd4       ?ProcessSetInterface@@YA?AW4CONTROL_RESPONSE@@PAUUFN_MDD_CONTEXT@@U_USB_DEVICE_REQUEST@@K@Z 10009bd4 f   usb_ufnmddbase_common_topaz_v1:enum.obj
 0001:00008d30       ?ProcessRequest@@YA?AW4CONTROL_RESPONSE@@PAUUFN_MDD_CONTEXT@@U_USB_DEVICE_REQUEST@@K@Z 10009d30 f   usb_ufnmddbase_common_topaz_v1:enum.obj
 0001:0000b7bc       doexit                     1000c7bc f   corelib0:cexit.obj
 0001:0000ba4c       CeLogMsg                   1000ca4c f   usb_usbfn_mx25_topaz_v1:i_pdd.obj
 0001:0000bb24       GetSetupPacket             1000cb24 f   usb_usbfn_mx25_topaz_v1:i_pdd.obj
 0001:0000bbec       InitQh0                    1000cbec f   usb_usbfn_mx25_topaz_v1:i_pdd.obj
 0001:0000bec4       PrimeQh0ForZeroTransfer    1000cec4 f   usb_usbfn_mx25_topaz_v1:i_pdd.obj
 0001:0000c104       HandleUSBReset             1000d104 f   usb_usbfn_mx25_topaz_v1:i_pdd.obj
 0001:0000c728       BuildTdBufferList          1000d728 f   usb_usbfn_mx25_topaz_v1:i_pdd.obj
 0001:0000f070       GetStringParam             10010070 f   usb_usbfn_os_mx25_topaz_v1:i_registry.obj
 0001:0000f1c0       GetMultiDWordParam         100101c0 f   usb_usbfn_os_mx25_topaz_v1:i_registry.obj
 0001:0000f384       GetBinParam                10010384 f   usb_usbfn_os_mx25_topaz_v1:i_registry.obj
 0001:0000f7b8       ??__E?_factory@?$singleton@V?$free_list@$0GE@Vallocator@ce@@@ce@@$03V?$static_allocator@V?$free_list@$0GE@Vallocator@ce@@@ce@@$03@2@@ce@@1Ulock_factory@12@A@@YAXXZ 100107b8 f   usb_ufnmddbase_common_topaz_v1:ufnmdd.obj
